:100000000C9458090C948D090C948D090C948D094D
:100010000C948D090C948D090C948D090C948D0908
:100020000C948D090C948D090C948D090C94521A22
:100030000C948D090C948D090C948D090C949816D0
:100040000C948D090C948D090C948D090C948D09D8
:100050000C9486420C94A9420C948D090C948D0941
:100060000C948D090C948D090C948D090C948D09B8
:100070000C948D090C948D090C948D090C948D09A8
:100080000C948D090C948D090C948D09436C656159
:1000900072696E67205374617473000A696E7661C9
:1000A0006C696420646174650A000A53657474693C
:1000B0006E67204D5050542062617420676F616CF0
:1000C0002025730A000A53657474696E67204D50C9
:1000D0005054204D6F64652025730A000A536574DF
:1000E00074696E6720457870657274204D6F646521
:1000F0002025730A0025642D253032643A253032DC
:10010000643A25303264004C6F61642020252D381C
:100110002E316620202020252D382E316620252DD9
:10012000382E316620202020252D382E31660049BA
:100130006E20202020252D382E31662020202025DD
:100140002D382E316620252D382E31662020202096
:10015000252D382E31660020202020202043686184
:100160007267652841682920205077722857292016
:1001700020205065616B5077722857292020456EEA
:100180006572677928576829206F76657220252E59
:1001900030662073656300252D362E326620252DAE
:1001A000342E32660A00252D362E326620252D3655
:1001B0002E326620252D362E326620252D362E3203
:1001C00066252D362E326620252D342E32662025CA
:1001D0002D352E31662025642025642025642025B8
:1001E0002D362E326620252D342E32660A000A5313
:1001F000657474696E67204C43442025730A006D52
:100200007070745F7363616E5F696E74657276613E
:100210006C3D2564206D696E0A20456E7465722000
:100220006E65773A20004F4B0A000A536574746973
:100230006E672041545820534220506F77657220DA
:1002400025730A000A53657474696E672041545817
:1002500020506F7765722025730A0041545820534F
:1002600069672E205057525F4F4B2025730A00417B
:100270005458205369672E2050535F4F4E2020253D
:10028000730A004154582050575220202020202526
:10029000730A0041545820534220505752202025C1
:1002A000730A004368616E6765204F7363696C6C05
:1002B00061746F722E204E6F77204F534343414C31
:1002C0003D25640A20456E746572206E65773A207C
:1002D0000020554252524C3D25642000204F53438C
:1002E00043414C3D2564200020556E7573656420A4
:1002F000737461636B203D25640020467573653A15
:100300002065653D253032782068663D253032789D
:10031000206C663D25303278206C623D2530327885
:10032000004D43553D2530366C7800252D31306C1D
:100330007520252D31306C7520252D31306C7520C0
:10034000252D31306C7520252D31306C7520252DF3
:1003500031306C7520252D31306C750A00565F697F
:100360006E3E4D617820202056206261743E4D61C2
:100370007820204120696E3E4D6178202020412068
:100380006C6F61643E4D61782054206261743E4D13
:100390006178202054206D69737320636E74204C43
:1003A000564420636E740A00446174652020202046
:1003B00020202054696D6520202020204261742077
:1003C000202020476F616C202020496E20202020B3
:1003D00020615F696E202050574D20207077725F3A
:1003E000696E20206D70707420207077722D6469A2
:1003F00066660A0044617465202020202020205475
:10040000696D652020202020416828696E29202000
:10041000204168286C6F61642920205028696E296A
:10042000202050286C6F61642920205128696E2992
:10043000202051286C6F6164290A00446174652092
:1004400020202020202054696D652020202020427B
:10045000617420202020476F616C202020496E208D
:1004600020202020615F696E202050574D202054AD
:100470005F426174207431202074322020765F6CDA
:100480006F616420615F6C6F61640A004375727212
:10049000656E742064656275673D3078255820204C
:1004A0004E65773A2000445F504F5745523D3078B3
:1004B00025780A00445F4C45443D307825780A0091
:1004C000445F4F573D307825780A00445F4D5050C7
:1004D000545F5343414E5F424553543D3078257835
:1004E0000A00445F4D5050545F5343414E3D3078B5
:1004F00025780A00445F4D5050543D307825780AE5
:1005000000445F4C4F41443D307825780A00445FF9
:100510004348415247453D307825780A00445F4FB3
:100520005045523D307825780A00456E746572203A
:100530004F6E2D426F6172642074656D702073651B
:100540006E736F72206964783A2000456E7465722C
:1005500020426174746572792074656D70207365D2
:100560006E736F72206964783A200042617474651A
:1005700072792054656D70203D2025352E3266003D
:10058000765F6C76645F687973743D25352E3266CC
:100590000A20456E746572206E65773A2000765F9A
:1005A0006C76643D25352E32660A20456E74657280
:1005B000206E65773A20004C6F616420637572721B
:1005C000656E74206C696D69743D25352E32660A3E
:1005D00020456E746572206E65773A2000496E7012
:1005E00075742063757272656E74206C696D6974C0
:1005F0003D25352E32660A20456E746572206E6583
:10060000773A2000765F676F616C5F6C6F61643D65
:1006100025352E32660A20456E746572206E657728
:100620003A2000765F676F616C3D25352E32660A91
:1006300020456E746572206E65773A2000666C7492
:100640005F666163746F723D25352E32660A204500
:100650006E746572206E65773A2000666C74206651
:100660006163746F7220636F6E74726F6C73207449
:10067000686520706572696F64206265666F726577
:10068000206E65787420626F6F7374207065726974
:100690006F640A00506C656173652073657420791E
:1006A0006F757220666978656420766F6C74616717
:1006B0006525730A000A53657474696E672046697C
:1006C00078656420566F6C74616765204D6F646552
:1006D0002025730A006174787320202D20736574BF
:1006E0002041545820534220706F77657220257343
:1006F0000A006174787020202D2041545820706FBA
:100700007765722025730A00727320202D20726590
:1007100073746F72652064656661756C74207365AF
:100720007474696E67730A0D006F7720202D206F37
:10073000772D6275732064756D700A0D006D6920E8
:10074000202D20736574204D505054207363616ECA
:1007500020696E74657276616C0A006D6220202DCE
:1007600020736574204D505054206261747465721A
:10077000792025730A006D7420202D207365742064
:100780004D5050542025730A006C7020202D20738A
:100790006574204C43442025730A00646920202D91
:1007A00020646973636F6E6E65637420696E707523
:1007B00074206D616E75616C6C790A0D006369203F
:1007C000202D20636F6E6E65637420696E70757482
:1007D000206D616E75616C6C790A0D00646C20206F
:1007E0002D20646973636F6E6E656374206C6F6136
:1007F00064206D616E75616C6C790A0D00636C200C
:10080000202D20636F6E6E656374206C6F616420B1
:100810006D616E75616C6C790A0D00762020202D5B
:100820002076657273696F6E0A0D00752020202D89
:1008300020757074696D650A0D00747320202D2079
:1008400074696D65207365740A0D00636320202D43
:100850002063686172676520737461747320636CD0
:100860006561720A0D00637320202D206368617238
:1008700067652073746174730A0D00742020202D45
:100880002074696D652073686F770A0D00646520B8
:10089000202D2064656275670A0D00737320202D7A
:1008A000207374617475732073756D6D6172790A4C
:1008B0000D00626D20202D206261747465727920B4
:1008C0007375626D656E750A0D00682020202D20FD
:1008D00068656C700A0D00756E6B6E6F776E2063C5
:1008E0006D640A006D2020202D206261636B2074EE
:1008F0006F206D61696E206D656E750A0D007268FE
:1009000020202D207265636F6E6E65637420687998
:10091000737465726573697320766F6C7461676553
:100920000A0D00647620202D20646973636F6E6E5B
:1009300065637420766F6C746167650A0D00766C70
:1009400020202D20766F6C74616765206C6F616468
:1009500020676F616C0A0D00666620202D20666C92
:100960006F617420706572696F6420666163746F73
:10097000720A0D00766720202D20766F6C746167F7
:100980006520676F616C0A0D00667620202D20625D
:1009900061747465727920666978656420766F6C1D
:1009A00074616765206D6F64650A0D0062612020C7
:1009B0002D206261747465727920766F6C74616742
:1009C0006520706172616D730A0D00746920202DBD
:1009D00020626174746572792073656E736F722022
:1009E0006F6E652D7769726520696E6465780A0D92
:1009F00000746520202D2062617474657279207402
:100A0000656D70657261747572650A0D00636120B1
:100A1000202D2063616C69627261746520766F6C51
:100A2000746167652072656164696E67730A0D00A1
:100A3000616C20202D206C696D6974206C6F61647D
:100A40002063757272656E740A0D00616920202D35
:100A5000206C696D697420696E707574206375729D
:100A600072656E740A0D00646520202D2064656235
:100A700075670A0D00682020202D2068656C700ABB
:100A80000D00426F6F737420566F6C746167652040
:100A9000617420323043203D25352E32660A2045D0
:100AA0006E746572204E65773A2000466C6F6174F3
:100AB00020566F6C7461676520617420323043206A
:100AC0003D25352E32660A20456E746572204E65CE
:100AD000773A2000496E2043757272656E743D2529
:100AE000352E32660A20456E74657220636F72720D
:100AF00065637465643A20004C6F616420437572CD
:100B000072656E743D25352E32660A20456E746519
:100B10007220636F727265637465643A20004C6F73
:100B2000616420566F6C746167653D25352E3266B1
:100B30000A20456E74657220636F72726563746516
:100B4000643A2000496E70757420566F6C7461674A
:100B5000653D25352E32660A20456E746572206328
:100B60006F727265637465643A20004261747465E3
:100B7000727920566F6C746167653D25352E32663B
:100B80000A20456E74657220636F727265637465C6
:100B9000643A20004C6F616420617665726167651C
:100BA0002063757272656E74203D25352E33662084
:100BB000410A004C6F616420766F6C746167652038
:100BC000676F616C203D25352E3166560A004D5009
:100BD0005054207363616E20696E74657276616C27
:100BE000203D2564206D696E0A004D5050542073DD
:100BF00063616E3A2050574D2075736564203D2027
:100C000025642C2062657374203D25642C20505788
:100C1000523D25352E33660A004D50505420765FE4
:100C2000626174203D25640A004D505054206C6F61
:100C3000636B2F6E6F6C6F636B203D256C752F257A
:100C40006C750A0054656D70206261747465727908
:100C5000203D25362E326620432028446566617586
:100C60006C74290A0054656D702073656E736F7221
:100C7000206572726F72203D256420430A0020288F
:100C800044656661756C7429205741524E494E4740
:100C90002074656D702073656E736F7220696420B7
:100CA0006E6F7420636F6E66696775726564005459
:100CB000656D702062617474657279203D25362EF1
:100CC0003266204300566F6C74616765206C6F61FB
:100CD00064207265636F6E6E656374206F66667301
:100CE0006574203D25352E326620560A00496E7007
:100CF0007574206973206D616E75616C6C79206408
:100D00006973636F6E6E65637465640A004C6F612E
:100D100064206C61737420646973636F6E6E6563C5
:100D200074656420004C6F6164206973206D616E8E
:100D300075616C6C7920646973636F6E6E65637442
:100D400065640A004C6F6164206973206C6F7720C2
:100D5000766F6C7461676520646973636F6E6E652E
:100D6000637465640A00566F6C74616765206C6F0C
:100D7000616420646973636F6E6E656374203D25E2
:100D8000352E316620560A004C6173742063686109
:100D900072676520004D6178206C6F616420637517
:100DA0007272656E74203D25352E316620410A0031
:100DB0004D617820696E7075742063757272656E0E
:100DC00074203D25352E316620410A00437572722C
:100DD000656E74206C6F6164203D25362E3366206D
:100DE000410A0043757272656E7420696E203D255C
:100DF000362E336620410A00566F6C746167652099
:100E00006C6F6164203D25352E326620560A0056EF
:100E10006F6C7461676520676F616C203D25352EAE
:100E20003166560A00566F6C7461676520666C6F98
:100E30006174203D25352E3166560A00566F6C745C
:100E400061676520626F6F7374203D25352E3166B2
:100E5000560A00566F6C7461676520696E203D25E7
:100E6000352E326620560A00566F6C746167652015
:100E7000626174203D25352E326620560A00566F79
:100E80006C7461676520636170203D25352E326684
:100E900020560A004C56442074696D652000557038
:100EA00074696D652000446174652000312E300D39
:100EB0000A00202573205374617274200052544339
:100EC0002025732C00436F7079726967687420481D
:100ED00065726A756C662055747665636B6C696EB5
:100EE000672C2055707073616C6120537765646561
:100EF0006E2C206865726A756C662E73650D0A002B
:100F00004669726D77617265205665722E20362EA5
:100F10003320323031332D30392D31350D0A002058
:100F2000252D382E316620252D382E316620252D91
:100F3000382E316620252D382E316620252D382E6D
:100F4000306620252D382E30660A004368617267AE
:100F5000652074696D6572206578706972656420BA
:100F60006166746572202575207365630A00426F9F
:100F70006F7374207265616368656420696E2025F3
:100F8000752073656320666C742D706572696F647B
:100F90002073657420746F202575207365630A00C3
:100FA000204D505054207363616E20646F6E653A1B
:100FB0002050574D2075736564203D202534642CE6
:100FC0002062657374203D2534642C205057523DB7
:100FD00025352E33660A00204D505054207363612E
:100FE0006E3A2050574D2075736564203D2025349E
:100FF000642C207363616E203D2534642C2050578F
:10100000523D25352E33660A0020252D362E3266B8
:1010100020252D362E326620252D362E32662025AF
:101020002D342E3266202534642020252D372E3392
:10103000662025642020252D372E3366200A0020C7
:10104000252D362E326620252D362E326620252D72
:10105000342E3266202534640A0020252D362E32A7
:101060006620252D362E326620252D362E3266201E
:10107000252D342E32662025346420252D352E3141
:101080006620256420256420256420252D362E32F7
:101090006620252D342E32660A00253034642D2535
:1010A0003032642D2530326420253032643A2530C8
:1010B00032643A2530326400745F626174203D20EE
:1010C00025362E32660A005761726E696E672E20D1
:1010D000426174746572792073656E736F722069F2
:1010E00064206E6F74207365740A005761726E69B4
:1010F0006E672E204E6F2074656D702073656E7361
:101100006F72730A00526573657474696E6700527A
:101110006573746F726520616C6C2073657474699B
:101120006E67733F20792F6E3A2000253034642D8E
:10113000253032642D2530326420253032643A2542
:101140003032643A253032640020257300204F6E1F
:101150002D426F617264002042617474657279007F
:101160002025362E32662000253032780025642076
:10117000000A006E616E00696E660000407A10F32E
:101180005A00A0724E18090010A5D4E80000E876B5
:1011900048170000E40B54020000CA9A3B0000000C
:1011A000E1F505000080969800000040420F000025
:1011B00000A08601000000102700000000E80300E6
:1011C0000000006400000000000A000000000001B0
:1011D00000000000002C76D888DC674F0823DFC1B0
:1011E000DFAE59E1B1B796E5E3E453C63AE651996B
:1011F0007696E8E6C28426EB898C9B62ED407C6F94
:10120000FCEFBC9C9F40F2BAA56FA5F490055A2A4A
:10121000F75C936B6CF9676DC11BFCE0E40D47FE56
:10122000F520E6B500D0ED902E030094357705004B
:1012300080841E080000204E0A000000C80C3333D2
:1012400033330F986E12831141EF8D2114893BE6E1
:101250005516CFFEE6DB18D1844B381BF77C1D906A
:101260001DA4BBE424203284725E228100C9F124D3
:10127000ECA1E53D27494E46494E4954594E414E51
:10128000CDCCCC3D0AD7233C17B7D13877CC2B3205
:101290009595E6241FB14F0A000020410000C84286
:1012A00000401C4620BCBE4CCA1B0E5AAEC59D74E5
:1012B000EAEBF3E085EC90E401C08193EF3FF9079E
:1012C000E0F3D9F311241FBECFEFD0E4DEBFCDBFD2
:1012D00084B78093B90314BE88E10FB6F894809365
:1012E0006000109260000FBE11E0A0E0B1E0E2E209
:1012F000F4EA00E00BBF02C007900D92A23CB107D8
:10130000D9F713E0A2ECB1E001C01D92A93BB107EF
:10131000E1F70E9410380C940F520C9400002091B9
:1013200070002C7F209370000097C1F081E08093C3
:10133000A6018091B60080628093B6001092B20040
:1013400082E08093B1008091B60090E08770907049
:101350000097C9F781E08093700008951092A6016C
:101360001092B2008091B6008F7D8093B60086E027
:101370008093B1008091B60090E0877090700097E4
:10138000C9F781E0809370000895AF92BF92CF9229
:10139000DF92EF92FF920F931F93CF93DF937B0126
:1013A0008C018DB79EB70A970FB6F8949EBF0FBEFB
:1013B0008DBFCDB7DEB7219685EF90E0EDB7FEB7D4
:1013C00092838183C801B70120E831E541E050E014
:1013D0000E94CB4A3B832A8330E1A32E3EE0B32E0A
:1013E000C12CD12CA60195010E94CB4A332727FDA1
:1013F00030953D832C83C801B701A60195010E9459
:10140000CB4A2CE3A22EB12CC12CD12CA6019501E4
:101410000E94CB4A332727FD30953F832E83C80196
:10142000B701A60195010E94CB4A772767FD709509
:10143000798768870E940B4E8DB79EB708960FB6C6
:10144000F8949EBF0FBE8DBF81E791E1EDB7FEB767
:10145000928381830E940B4E0F900F90DF91CF916A
:101460001F910F91FF90EF90DF90CF90BF90AF90C2
:101470000895EAEBF3E080E4EF3FF80709F0A8F401
:1014800020E030E005C080E4EF3FF80709F058F4B1
:1014900031968081853CB9F72F5F3F4F80E4EF3F65
:1014A000F807B1F3A8F3C901089520E030E0FBCFBD
:1014B000009749F4109246011092C2010A9A1298BC
:1014C000089A1098089581E0809346010898109A30
:1014D0000895009739F40A9A12981092C201229A3C
:1014E0002A98089522982A9A08956F927F928F924F
:1014F0009F92AF92BF92CF92DF92EF92FF920F93A3
:101500001F93DF93CF93CDB7DEB729970FB6F8942B
:10151000DEBF0FBECDBF1092D7018FEF89837CE372
:10152000C72E72E0D72EEE24FF24882462E0A62E78
:10153000B12CAC0EBD1E3E010894611C711C8E01C5
:10154000065F1F4F9E2CC301B5010E949740898101
:101550008F3F09F485C08E3F09F482C0C5010E9407
:10156000B240F6018087F501D701AA0FBB1FAA0F71
:10157000BB1FAA0FBB1FAE0DBF1DA45CBD4F819149
:101580008D93E017F107D9F79091B802F6018081A9
:101590009817D1F193948981882369F00894E11C0C
:1015A000F11C89E090E0C80ED91E98E0E916F1041C
:1015B00049F648E0942E882089F48FEF8093B80292
:1015C0008093B9028093BA028093BB028093BC02DD
:1015D0008093BD028093BE028093BF02892D29961D
:1015E0000FB6F894DEBF0FBECDBFCF91DF911F9134
:1015F0000F91FF90EF90DF90CF90BF90AF909F90B2
:101600008F907F906F9008959091B9028181981783
:1016100009F69091BA028281981709F0BBCF909198
:10162000BB028381981709F0B5CF9091BC028481E9
:10163000981709F0AFCF9091BD028581981709F0F6
:10164000A9CF9091BE028681981709F0A3CF9091FF
:10165000BF028781981709F09DCF882483949ACF81
:101660008093D701A8CF0E94750A8093D601089570
:1016700000D081E791E1EDB7FEB7928381830E94AC
:101680000B4E0F900F9008952F923F924F925F92C2
:101690006F927F928F929F92AF92BF92CF92DF9282
:1016A000EF92FF920F931F93CF93DF930E94330B20
:1016B0008091D601882309F4BEC0CCE3D2E0AA24ED
:1016C000BB24BDE64B2EB1E15B2EA8E6CA2EA1E1FC
:1016D000DA2EF0E62F2EF1E13F2E00D000D0ADB78C
:1016E000BEB712965C924E9211971496BC92AE922F
:1016F00013970E940B4E0F900F900F900F90850143
:10170000000F111F000F111F000F111F0A0D1B1DCD
:10171000045C1D4FC8010E94F741FC01BF018827EE
:1017200077FD8095982F0E9481493B014C017801FB
:1017300000E010E0D7018D917D0100D000D0EDB721
:10174000FEB73196ADB7BEB71296DC92CE92119726
:10175000828313820E940B4E0F5F1F4F0F900F90DA
:101760000F900F900830110529F700D000D000D05D
:101770000DB71EB70F5F1F4FEDB7FEB73282218244
:10178000662D772D882D992D20E030E048EC52E42D
:101790000E94E648D80112966D937D938D939C9399
:1017A00015970E940B4E888129813A81EB817C81BB
:1017B0006D815E814F81ADB7BEB716960FB6F894B6
:1017C000BEBF0FBEADBF9091B802981709F47AC0A2
:1017D00090911403981709F444C088858823F1F187
:1017E00080E091E000D000D0E9E4F1E1ADB7BEB710
:1017F0001296FC93EE93119714969C938E931397E5
:101800000E940B4E0F900F90E1E7F1E1ADB7BEB72C
:101810001296FC93EE9311970E940B4E0894A11C14
:10182000B11C29968091D60190E00F900F90A816D8
:10183000B9060CF452CFDF91CF911F910F91FF9019
:10184000EF90DF90CF90BF90AF909F908F907F9060
:101850006F905F904F903F902F90089589E091E0B6
:10186000C1CF80911503821709F0B7CF809116037D
:10187000831709F0B2CF809117038E1709F0ADCF0F
:1018800080911803871709F0A8CF80911903861754
:1018900009F0A3CF80911A03851709F09ECF80919C
:1018A0001B03841709F099CF00D0EDE4F1E1ADB747
:1018B000BEB71296FC93EE9311970E940B4E0F90B9
:1018C0000F908BCF9091B902921709F081CF909130
:1018D000BA02931709F07CCF9091BB029E1709F0D2
:1018E00077CF9091BC02971709F072CF9091BD020B
:1018F000961709F06DCF9091BE02951709F068CF49
:101900009091BF02941709F063CF00D027E531E131
:10191000EDB7FEB7328321830E940B4E8881298167
:101920003A81EB817C816D815E814F810F900F90B8
:101930004FCFEAE7F0E080E8808380818760808392
:1019400010927B0088EF80937E0080818860808386
:10195000808180648083089580937C0080917C00E6
:10196000806C80937C0086E080937A0080917A007E
:10197000806880937A0080917A00806480937A00F6
:1019800080917A0086FDFCCF88E090E060E070E016
:1019900020917A00206420937A0020917A0026FD1D
:1019A000FCCF2091780030917900620F731F01976E
:1019B00079F780917A008F7780937A007695679592
:1019C000769567957695679580E090E00E947F49CF
:1019D0000895CF92DF92EF92FF920F931F93CF93D0
:1019E000DF937B018C016A01E901FA018081882380
:1019F00071F4C801B70120E030E0A9010E94314A2A
:101A000018160CF054C064971092FE010CC0C80167
:101A1000B70120E030E0A9010E94314A181604F510
:101A200064961092FE018091E9019091EA01A091E3
:101A3000EB01B091EC010196A11DB11D8093E9016C
:101A40009093EA01A093EB01B093EC01CE01DF91FA
:101A5000CF911F910F91FF90EF90DF90CF9008955D
:101A6000C801B70120E030E0A9010E94E24887FDEB
:101A700031C08091FE018F5F8093FE01823098F229
:101A800081508093FE018091E5019091E601A09143
:101A9000E701B091E8010196A11DB11D8093E50118
:101AA0009093E601A093E701B093E801CFCFC8017E
:101AB000B70120E030E0A9010E94E24887FFD9CFBA
:101AC00081E0F601808364968091FE018F5F8093B0
:101AD000FE01D4CF6497F60110828091FE018F5FE2
:101AE0008093FE01CBCFEF92FF920F931F93CF9382
:101AF000DF93609110037091110380911203909114
:101B000013032091FC023091FD024091FE0250919E
:101B1000FF020E94314A18160CF580919A019091AB
:101B20009B0123E08F3F920728F580919A019091C5
:101B30009B01E0919C01F0919D019093990180930C
:101B40009801809198019091990191838083DF9110
:101B5000CF911F910F91FF90EF9008958091DE013A
:101B6000882359F080919A0190919B0133E08F3F37
:101B70009307D8F28FEF93E0DCCF60910C03709164
:101B80000D0380910E0390910F03E0907101F0908E
:101B900072010091730110917401A80197010E94D4
:101BA000314A18160CF063C060910C0370910D035C
:101BB00080910E0390910F03A80197010E947D4828
:101BC00020E030E0A9010E94314A18160CF057C0FD
:101BD00060910C0370910D0380910E0390910F039F
:101BE000A80197010E947D4820E030E048E452E4DB
:101BF0000E94354A0E945349809198019091990121
:101C0000860F971F97FDF6C020919A0130919B0196
:101C10002817390720F480919A0190919B01E09157
:101C20009C01F0919D01909399018093980180917E
:101C3000980190919901918380838091A002909165
:101C4000A102A091A202B091A3020196A11DB11D13
:101C50008093A0029093A102A093A202B093A3024A
:101C6000DF91CF911F910F91FF90EF900895809198
:101C7000FD011816D4F481508093FD0168CF609166
:101C80000C0370910D0380910E0390910F03A80136
:101C900097010E947D48905820E030E048E452E4EB
:101CA0000E94354A0E945349A7CF8091FB01909131
:101CB000FC0101969093FC018093FB0180918C02C2
:101CC00090918D02A0918E02B0918F0280930803B3
:101CD00090930903A0930A03B0930B0380918B01A7
:101CE000882309F4A6C060911003709111038091BC
:101CF00012039091130320910C0330910D03409136
:101D00000E0350910F030E94354A9B01AC012093B2
:101D10008C0230938D0240938E0250938F0260911B
:101D20006101709162018091630190916401209141
:101D300010033091110340911203509113030E943C
:101D40007D4820E030E0A9010E94314A18160CF0CD
:101D500054C0609161017091620180916301909122
:101D600064012091100330911103409112035091AE
:101D700013030E947D4820E030E048E452E40E94D2
:101D8000354A0E945349E62EE7017E01F72EE7010E
:101D9000CF31D10510F0CEE1D0E06091FC0270911E
:101DA000FD028091FE029091FF02E0901003F090FE
:101DB000110300911203109113032DEC3CEC4CE441
:101DC0005EE30E947D48A80197010E94314A1816DF
:101DD000CCF180919801909199018C0F9D1F97FDF6
:101DE000FFC020919A0130919B012817390708F410
:101DF0009CCE9FCE80E090E012CF60916101709107
:101E000062018091630190916401209110033091EF
:101E1000110340911203509113030E947D48905882
:101E200020E030E048E452E40E94354A0E945349E1
:101E3000AACF6091FC027091FD028091FE02909108
:101E4000FF0259CF6091100370911103809112032A
:101E500090911303209161013091620140916301DF
:101E6000509164010E94314A18169CF580919801A6
:101E7000909199018C0F9D1F97FDB5C020919A01FB
:101E800030919B012817390720F480919A01909195
:101E90009B01E0919C01F0919D01909399018093A9
:101EA000980180919801909199019183808360912C
:101EB000B4027091B5028091B6029091B70220E011
:101EC00030E0A9010E94E24887FF41CE1092D10183
:101ED0003ECE609110037091110380911203909196
:101EE000130320916101309162014091630150918F
:101EF00064010E94E24887FF2ACE80918A018823EC
:101F000009F466C08091D101882309F4DFC0609193
:101F10008C0270918D0280918E0290918F0220919F
:101F2000B4023091B5024091B6025091B7020E94BE
:101F3000314A18160CF4B1C02091F9013091FA0120
:101F40002115310509F052C08091980190919901B5
:101F500090933B0280933A0284E690E03093C4026F
:101F60002093C3029093FA018093F90120919A0182
:101F700030919B012817390720F480919A019091A4
:101F80009B01E0919C01F0919D01909399018093B8
:101F9000980180919801909199019183808380911B
:101FA0008C0290918D02A0918E02B0918F0280934D
:101FB0001E0390931F03A0932003B09321038091ED
:101FC0001D03886080931D0387E08093FD01BFCDD2
:101FD00080919801909199018C1B9D0B97FF01CFE7
:101FE00080E090E0A6CD80E090E053CFC9018C590D
:101FF0009F4F43E08F3F940708F4B0CF1092D10178
:102000008091C1029091C20297FDB7C020919A01C0
:1020100030919B012817390720F480919A01909103
:102020009B01E0919C01F0919D0190939901809317
:10203000980180919801909199019183808380917A
:10204000B4029091B502A091B602B091B70280930C
:102050001E0390931F03A0932003B093210380E0FD
:1020600090E0A0E8BFEB8093B4029093B502A093F8
:10207000B602B093B7028091C1029091C2029093D0
:10208000C4028093C3021092FA011092F901809168
:102090001D03806180931D0397CF2091F90130913A
:1020A000FA013093C2022093C10280918C02909178
:1020B0008D02A0918E02B0918F028093B402909312
:1020C000B502A093B602B093B7023ACF85E08093F1
:1020D000FD0160918C0270918D0280918E02909131
:1020E0008F02209108033091090340910A03509117
:1020F0000B03C0919801D09199010E947D484BEA51
:1021000051E09E010E94E90C9093990180939801FF
:10211000809198019091990123E08F3F920734F1CB
:102120006091100370911103809112039091130339
:10213000E0906101F09062010091630110916401EF
:102140002DEC3CEC4CE45EE30E947E48A801970134
:102150000E94E24887FF14C08091C1029091C202A0
:1021600090939901809398011092AB01809198010E
:102170009091990197FD34CF34CE80E090E051CF1B
:102180008FEF93E09093990180939801EFCFCF92D6
:10219000DF92EF92FF920F931F93CF93DF936091A3
:1021A00090027091910280919202909193022091FD
:1021B00075013091760140917701509178010E942C
:1021C000314A1816ECF580918C0190918D01845361
:1021D0009F4F97FDBDC020918E0130918F01281730
:1021E000390720F480918E0190918F01E091900148
:1021F000F091910190938D0180938C0180918C01DD
:1022000090918D01918380838091A4029091A50289
:10221000A091A602B091A7020196A11DB11D8093C5
:10222000A4029093A502A093A602B093A702DF9107
:10223000CF911F910F91FF90EF90DF90CF90089575
:102240008091DD018823E1F080918E0190918F01D2
:1022500023E08F3F920708F07EC080918E0190911D
:102260008F01E0919001F091910190938D01809305
:102270008C0180918C0190918D0191838083D7CFC7
:102280008091DC01882301F7E0906501F090660100
:10229000009167011091680120912E0230912F0268
:1022A0004091300250913102C801B7010E947D482F
:1022B00020E030E0A9010E94314A18160CF068C0F5
:1022C00020912E0230912F02409130025091310224
:1022D000C801B7010E947D4820E030E048E452E4A4
:1022E0000E94354A0E945349C62EE6016E01D72E40
:1022F000E601C430D10510F0C3E0D0E020912E02F9
:1023000030912F024091300250913102C801B70143
:102310000E94E24887FF22C080918C0190918D013C
:102320008C0F9D1F33E08D3F930708F047C08091CD
:102330008C0190918D018C0F9D1F97FD26C02091DF
:102340008E0130918F012817390708F486CF89CF85
:1023500080E090E04BCF8FEF93E083CF20912E026F
:1023600030912F024091300250913102C801B701E3
:102370000E94314A18160CF05ACF80918C0190912E
:102380008D018C1B9D0B97FFDACF80E090E069CF29
:1023900020912E0230912F02409130025091310253
:1023A000C801B7010E947D48905820E030E048E421
:1023B00052E40E94354A0E94534996CF80918C0185
:1023C00090918D01CCEFD3E0C81BD90BB0CF94B165
:1023D000936094B995B1936095B9833081F084305E
:1023E00038F0863091F0873039F0853041F008952B
:1023F000813021F0823028F0299808952998289872
:10240000089585B1836085B90895299885B1817053
:1024100085B90895CF93DF938CE192E020911C025F
:1024200030911D02FC013197A081FC01329770812F
:10243000FC0133976081FC01349750810597EC01D2
:102440004881EDB7FEB73E970FB6F894FEBF0FBEBA
:10245000EDBF31968BE291E1CDB7DEB79A838983E8
:1024600033832283A4831582768317826087118643
:1024700052871386448715860E940B4EEDB7FEB730
:102480003E960FB6F894FEBF0FBEEDBFDF91CF9121
:102490000895A7E1B2E0E6EAF3E087E001900D924B
:1024A0008150E1F70895CF93DF93ECE9F1E0A0913B
:1024B0009C01B0919D01EF01229788819981349709
:1024C000918380838081918111969C938E935D98F6
:1024D000DF91CF910895E0E8F0E020EC20832081A7
:1024E000236020832AE020938100A8E8B0E01196C1
:1024F0009C938E938D919C911197559A80818063C6
:1025000080838FEF91E090938D0180938C01909365
:102510008B0080938A00549A81E080936F008FEF44
:1025200093E090938F0180938E0190939B01809311
:102530009A01789408958FEF81B911B812B884B9CF
:1025400014B815B887B917B818B88AB91AB81BB82B
:102550000F980E980D980C980B9888EF80937E003A
:10256000399A419A389A409A579A5F9A8091C40151
:1025700081FF0BC080914701882309F4CAC081E024
:1025800090E00E94690A8091C40180FF09C0809197
:102590004601882309F0C4C080E090E00E94580AF8
:1025A00081E090E00E948F0981E791E06DE270E0A8
:1025B00044E050E00E94C04E85E791E061E370E0A6
:1025C00044E050E00E94C04E89E791E066E370E08D
:1025D00044E050E00E94C04E81E691E06DE170E081
:1025E00044E050E00E94C04E85E691E061E270E078
:1025F00044E050E00E94C04E89ED91E065E370E058
:1026000041E050E00E94C04E88EB92E064E470E04C
:1026100049E050E00E94C04E84E193E06DE470E038
:1026200049E050E00E94C04E88E591E06CE070E027
:1026300044E050E00E94C04E8CE591E060E170E023
:1026400044E050E00E94C04E85EC91E064E170E00F
:1026500044E050E00E94C04E89EC91E068E170E0F7
:1026600044E050E00E94C04E80E591E064E070E0FC
:1026700044E050E00E94C04E84E591E068E070E0E4
:1026800044E050E00E94C04E8CE491E060E070E0D5
:1026900044E050E00E94C04E8DE791E06AE370E0B4
:1026A00044E050E00E94C04E89E691E065E270E0AF
:1026B00044E050E00E94C04E8DE691E069E270E097
:1026C00044E050E00E94C04E82E891E06EE370E08A
:1026D00044E050E00E94C04E8AE891E062E470E07D
:1026E00044E050E00E94C04E8BE891E063E470E06B
:1026F00044E050E00E94C04E80E691E06CE170E062
:1027000041E050E00E94C04E8FEF93E00E946B12B8
:10271000089580E090E00E94690A8091C40135CF5D
:1027200081E090E00E94580A3BCFEF92FF920F9316
:102730001F93CF93DF938091D601882309F4ADC016
:102740008091B8028F3F09F456C088EB92E00E9456
:10275000F7419C01B901882777FD8095982F0E9449
:10276000814920E030E048EC52E40E94E648E62E41
:10277000F72E082F192F2091D2013091D30126FD79
:10278000B7C0C801B70120E030E048EA52E40E9437
:10279000314A1816FCF41092D6018091A80290914B
:1027A000A902A091AA02B091AB020196A11DB11D90
:1027B0008093A8029093A902A093AA02B093AB02BF
:1027C0000F2EF0E0EF2EF0E0FF2EF8EC0F2FF1E4EB
:1027D0001F2FF02DF894E0924801F09249010093E8
:1027E0004A0110934B017894DF91CF911F910F9183
:1027F000FF90EF9008958091B9028F3F09F0A5CF27
:102800008091BA028F3F09F0A0CF8091BB028F3F29
:1028100009F09BCF8091BC028F3F09F096CF809149
:10282000BD028F3F09F091CF8091BE028F3F09F02A
:102830008CCF8091BF028F3F09F087CF8091A80293
:102840009091A902A091AA02B091AB020196A11D9C
:10285000B11D8093A8029093A902A093AA02B093FD
:10286000AB028091D2019091D30186FF36C000D097
:1028700087EC90E1EDB7FEB7928381830E940B4E07
:102880000F900F900F2EF0E0EF2EF0E0FF2EF8ECFF
:102890000F2FF1E41F2FF02D9DCF0E94330B80915D
:1028A000D601882309F04CCF8091A8029091A9020B
:1028B000A091AA02B091AB020196A11DB11D809317
:1028C000A8029093A902A093AA02B093AB028091B0
:1028D000D2019091D30186FD2AC00F2EF0E0EF2E99
:1028E000F0E0FF2EF8EC0F2FF1E41F2FF02D72CF48
:1028F00000D000D000D028EB30E1CDB7DEB73A836E
:102900002983262F372F482F592FEDB7FEB7238362
:102910003483458356830E940B4E2DB73EB72A5F02
:102920003F4F0FB6F8943EBF0FBE2DBF2ACF00D049
:102930008BEE90E1CDB7DEB79A8389830E940B4E70
:102940000F900F900F2EF0E0EF2EF0E0FF2EF8EC3E
:102950000F2FF1E41F2FF02D3DCF6091DF0170911B
:10296000E0016115710551F481E090E09093E00180
:102970008093DF0168E873E1CB01089588E893E173
:102980000E94A44A61157105B9F761E070E0CB01BE
:102990000895CF93DF93C091DF01D091E00120979C
:1029A000E9F0BE0180E090E00E947F499B01AC010C
:1029B00060918201709183018091840190918501E1
:1029C0000E94E6480E945349262F372F2C173D07B7
:1029D00008F49E01C901DF91CF91089581E090E054
:1029E0009093E0018093DF0120E030E040E85FE376
:1029F000C1E0D0E0DDCF2F923F924F925F926F9275
:102A00007F928F929F92AF92BF92CF92DF92EF927E
:102A1000FF920F931F93DF93CF9300D000D0CDB7D9
:102A2000DEB73B014C0120914801309149014091B2
:102A30004A0150914B0160E070E080EA91E40E940D
:102A40007D4826EA3BE944EC5CE30E94354A20914C
:102A50006D0130916E0140916F01509170010E94A3
:102A60007E48F62E072F182FE92E862F902FA12FA4
:102A7000BE2D89839A83AB83BC832091480130911A
:102A8000490140914A0150914B0160E070E080EAB9
:102A900091E40E947D4826EA3BE944EC5CE30E9415
:102AA000354A2091690130916A0140916B01509142
:102AB0006C010E947E485B016C0115012601C40176
:102AC000B3012F2D302F412F5E2D0E94314A87FDFB
:102AD00007C08091F7019091F801009709F49DC01B
:102AE0008091860190918701009709F05CC08091E8
:102AF0001D03806480931D038091DF019091E001AC
:102B00009093E2018093E1018091F7019091F801A7
:102B10008130910559F08091F3019091F401019673
:102B20009093F4018093F30180FD63C020926101D2
:102B300030926201409263015092640160916101A0
:102B40007091620180916301909164012091FC0277
:102B50003091FD024091FE025091FF020E94314AE5
:102B60001816C4F58CE390E090938701809386015A
:102B70008091F5019091F601009709F447C02092E9
:102B8000610130926201409263015092640110929F
:102B9000F6011092F5011092E0011092DF011092FF
:102BA000F8011092F7010F900F900F900F90CF91B6
:102BB000DF911F910F91FF90EF90DF90CF90BF902A
:102BC000AF909F908F907F906F905F904F903F90CD
:102BD0002F90089588E790E0909387018093860175
:102BE0001092E0011092DF011092F8011092F701AB
:102BF000DACF89819A81AB81BC8180936101909306
:102C00006201A0936301B093640198CF81E090E0EA
:102C10009093F6018093F501E3CFA0926101B09209
:102C20006201C0926301D09264010E94C914909322
:102C30008701809386019093E4018093E301809162
:102C4000DF019091E0019093E2018093E101809196
:102C50001D03806280931D031092E0011092DF013A
:102C600081E090E09093F8018093F7019CCFAF92C0
:102C7000BF92CF92DF92EF92FF920F931F938091BA
:102C8000DA019091DB01009721F5609110037091BA
:102C900011038091120390911303E0907901F09059
:102CA0007A0100917B0110917C01A80197010E949B
:102CB000E24887FF17C08091DC01882399F1809159
:102CC0008101882331F488E790E09093DB018093C1
:102CD000DA011F910F91FF90EF90DF90CF90BF909E
:102CE000AF900895A0901003B0901103C09012030C
:102CF000D0901303C801B70120917D0130917E016E
:102D000040917F01509180010E947E48A60195016B
:102D10000E94E24887FFDDCF1092DC018AE08093B9
:102D20008101D7CF80918101815080938101C9CFEA
:102D30001F920F920FB60F920BB60F921124EF92C3
:102D4000FF920F931F932F933F934F935F936F9334
:102D50007F938F939F93AF93BF93EF93FF93809154
:102D6000A9019091AA0101979093AA018093A901CA
:102D7000009709F001C16091FC027091FD02809101
:102D8000FE029091FF0220911003309111034091B7
:102D90001203509113030E94314A18160CF403C118
:102DA00010E0409887E00E94AC0C209150013091D7
:102DB000510140915201509153010E94354A9B01AB
:102DC000AC012093100330931103409312035093EE
:102DD000130360911003709111038091120390917D
:102DE000130320E030E048ED51E40E94314A181608
:102DF0009CF480919C0290919D02A0919E02B091C2
:102E00009F020196A11DB11D80939C0290939D028B
:102E1000A0939E02B0939F0286E00E94AC0C20918A
:102E20004C0130914D0140914E0150914F010E9453
:102E3000354A9B01AC012093FC023093FD02409384
:102E4000FE025093FF026091FC027091FD0280919E
:102E5000FE029091FF0220E030E048ED51E40E9434
:102E6000314A18169CF48091980290919902A09191
:102E70009A02B0919B020196A11DB11D8093980208
:102E800090939902A0939A02B0939B020E94730DB3
:102E90008091A0019091A101A091A201B091A30104
:102EA0000196A11DB11D8093A0019093A101A09353
:102EB000A201B093A301112309F09CC0419A83E0C1
:102EC0000E94AC0C20915C0130915D0140915E014B
:102ED00050915F010E94354A2091C40123FF6EC0CA
:102EE00020E030E040E250E40E947D482DEC3CECD4
:102EF0004CEC5DE30E94E6487B018C016E2D7F2D3A
:102F0000802F912F2091C5013091C6014091C701BA
:102F10005091C8010E947D489B01AC012093900212
:102F2000309391024093920250939302409A85E02D
:102F30000E94AC0C209154013091550140915601F2
:102F4000509157010E94354A9B01AC0120932E02FB
:102F500030932F0240933002509331020E94C710E9
:102F6000A89585E090E09093AA018093A9018091B3
:102F70001D03816080931D03FF91EF91BF91AF917D
:102F80009F918F917F916F915F914F913F912F9181
:102F90001F910F91FF90EF900F900BBE0F900FBEFF
:102FA0000F901F90189510921E0210921F021092FF
:102FB000200210922102419811E0F3CE20E030E08F
:102FC00040E05FE30E947D4829EA37E848E05EE39D
:102FD0000E94E6487B018C017F2D912F20E030E09C
:102FE000A9010E94E24887FF89CFEE24FF2400E078
:102FF00010E084CF80910C0390910D03A0910E03FB
:10300000B0910F038093360290933702A093380259
:10301000B093390284E00E94AC0C209158013091A9
:10302000590140915A0150915B010E94354A20E0BC
:1030300030E040E05FE30E947D4829EA37E848E05D
:103040005EE30E94E6487B018C017F2D912F20E0FA
:1030500030E0A9010E94E24887FF04C0EE24FF246B
:1030600000E010E06E2D7F2D802F912F2091C9015F
:103070003091CA014091CB015091CC010E947D4812
:103080009B01AC0120930C0330930D0340930E037E
:1030900050930F0313CFEF92FF920F931F93609102
:1030A000FF0170910002809101029091020220E0E4
:1030B00030E0A9010E947E48209103023091040271
:1030C00040910502509106020E947E48209107021D
:1030D000309108024091090250910A020E947E48F4
:1030E00020910B0230910C0240910D0250910E0282
:1030F0000E947E487B018C0120910F0230911002CA
:103100004091110250911202CA01B9012E2D3F2D9A
:10311000402F512F0E947E4820E030E040EA50E4EA
:103120000E94E6481F910F91FF90EF900895A091A3
:10313000C9028A2F65E00E94984AE92FF0E02091A9
:103140009002309191024091920250919302EE0FC1
:10315000FF1FEE0FFF1FE150FE4F2083318342839C
:103160005383AF5FA093C90280918A01882379F0CD
:103170008091F20160916001982F9F5F9093F2011E
:103180000E94984A992319F481E08093D10108950F
:10319000AF92BF92CF92DF92EF92FF920F931F9365
:1031A0008091F101982F9F5F9093F1016CE30E9451
:1031B000984A992309F44EC18091D901882309F4D2
:1031C0003EC18091C4018370833029F4809146010F
:1031D000882309F045C1809186019091870101976C
:1031E00090938701809386018091DF019091E001A7
:1031F00001969093E0018093DF016091CD01709181
:10320000CE018091CF019091D00120E030E040E8E4
:103210005FE30E947E486093CD017093CE0180935E
:10322000CF019093D0016091FC027091FD028091DA
:10323000FE029091FF0220910C0330910D0340910A
:103240000E0350910F030E94354A7B01082FB92EBF
:10325000862F9F2DA02FBB2D8093880290938902EB
:10326000A0938A02B0938B026E2D7F2D802F9B2D11
:103270002091C5023091C6024091C7025091C80208
:103280000E94314A181664F48E2D9F2DA02FBB2D5D
:103290008093C5029093C602A093C702B093C80260
:1032A00060912E0270912F02809130029091310234
:1032B000209190023091910240919202509193029C
:1032C0000E94354A162FD72EC82EA92E862F9D2D47
:1032D000AC2DBA2D8093000390930103A0930203B9
:1032E000B0930303612F7D2D8C2D9A2D20913202F6
:1032F0003091330240913402509135020E94314A9C
:10330000181664F4812F9D2DAC2DBA2D80933202B6
:1033100090933302A0933402B0933502609113026C
:103320007091140280911502909116022E2D3F2D5E
:10333000402F5B2D0E947E4860931302709314020D
:103340008093150290931602609104037091050317
:103350008091060390910703212F3D2D4C2D5A2D6E
:103360000E947E48609304037093050380930603D4
:103370009093070320910C0330910D0340910E03AD
:1033800050910F03609122027091230280912402D8
:10339000909125020E947E4860932202709323023E
:1033A0008093240290932502209190023091910203
:1033B000409192025091930260912A0270912B02E7
:1033C00080912C0290912D020E947E4860932A02E7
:1033D00070932B0280932C0290932D028091DA013E
:1033E0009091DB01009711F101979093DB0180939D
:1033F000DA010097D9F48091DC01882309F44FC0E9
:1034000081E08093DC018091AC029091AD02A091AB
:10341000AE02B091AF020196A11DB11D8093AC0226
:103420009093AD02A093AE02B093AF021F910F91A3
:10343000FF90EF90DF90CF90BF90AF900895609194
:1034400010037091110380911203909113030E9455
:10345000FB14B7CE81E08093F1010E949718ACCEA7
:1034600080914701882309F4B6CE8091C201882358
:1034700009F0B1CE8091A80181508093A8018823E2
:1034800009F0A9CE81E08093C2010A9A129A83E0E2
:103490008093A8018AE091E00E942B4E9CCE0E946E
:1034A0004912AECF1F920F920FB60F920BB60F922A
:1034B00011242F933F934F935F936F937F938F9339
:1034C0009F93AF93BF93EF93FF9380911D0382600F
:1034D00080931D032091A601222341F480E1809373
:1034E000B2008091A7018F5F8093A701809188012E
:1034F00090918901181619067CF4809188019091A9
:1035000089010197909389018093880180918801B6
:1035100090918901009719F12223D1F08091A701A0
:1035200081508093A701882301F1FF91EF91BF9112
:10353000AF919F918F917F916F915F914F913F914B
:103540002F910F900BBE0F900FBE0F901F901895EC
:103550008091A701813149F71092A70109C080E04D
:103560000E94E7112091A601D7CF80E18093A701A7
:103570008091940290919502A0919602B091970249
:103580000196A11DB11D8093940290939502A09382
:103590009602B09397020E949E430E94C8188091A1
:1035A0001E0290911F02A0912002B091210201966B
:1035B000A11DB11D80931E0290931F02A0932002B3
:1035C000B09321028091DC01882309F4AECF809171
:1035D000260290912702A0912802B091290201961B
:1035E000A11DB11D8093260290932702A09328026B
:1035F000B09329029ACFCF93DF938BEA93E0209187
:10360000AB033091AC03FC013197A081FC013297F0
:103610007081FC0133976081FC01349750810597DC
:10362000EC014881EDB7FEB73E970FB6F894FEBFA8
:103630000FBEEDBF31968AE990E1CDB7DEB79A8330
:10364000898333832283A4831582768317826087DC
:10365000118652871386448715860E940B4EEDB75C
:10366000FEB73E960FB6F894FEBF0FBEEDBFDF91DA
:10367000CF9108952F923F924F925F926F927F92D7
:103680008F929F92AF92BF92CF92DF92EF92FF9272
:103690000F931F93DF93CF93CDB7DEB72E970FB65F
:1036A000F894DEBF0FBECDBFE090EF01F090F001C7
:1036B0000894E11CF11CF092F001E092EF01C701C7
:1036C0008F709070009789F4609148017091490162
:1036D00080914A0190914B0120E030E040E252E4B9
:1036E0000E94314A18160CF47AC08091D201909150
:1036F000D30180FF07C02FE0E222FF24E114F10490
:1037000009F426C18091D2019091D30182FF09C0B2
:103710008091EF019091F0018F709070009709F403
:10372000B7C18091D2019091D30183FF09C08091EC
:10373000EF019091F0018F709070009709F4F0C143
:103740008091D2019091D30184FF04C080911D0328
:1037500083FD88C28091D2019091D30185FF04C07E
:1037600080911D0384FDBEC28091D2019091D3014E
:1037700081FF04C080911D0385FDF4C28091D201B8
:103780009091D30181FF04C080911D0386FDC2C0CA
:103790008091D2019091D30190FF08C08091EF01F8
:1037A0009091F0018F709070009769F12E960FB68E
:1037B000F894DEBF0FBECDBFCF91DF911F910F9167
:1037C000FF90EF90DF90CF90BF90AF909F908F9041
:1037D0007F906F905F904F903F902F9008958091D1
:1037E000B0029091B102A091B202B091B3020196E1
:1037F000A11DB11D8093B0029093B102A093B202BB
:10380000B093B30272CF0E94FB1AEDB7FEB77A975E
:103810000FB6F894FEBF0FBEEDBFEDB6FEB608942E
:10382000E11CF11C8FE19FE0928381836091220271
:1038300070912302809124029091250220E030E0D3
:1038400041E655E40E94E648D70112966D937D93B8
:103850008D939C93159760912A0270912B02809111
:103860002C0290912D0220E030E041E655E40E94C8
:10387000E648F70166837783808791878091880285
:1038800090918902A0918A02B0918B0282879387DE
:10389000A487B5878091000390910103A091020352
:1038A000B091030386879787A08BB18B6091130239
:1038B00070911402809115029091160220E030E080
:1038C00041E655E40E94E648D70152966D937D93F8
:1038D0008D939C935597609104037091050380919B
:1038E00006039091070320E030E041E655E40E9492
:1038F000E648F701668B778B808F918F0E940B4E85
:103900002DB73EB7265E3F4F0FB6F8943EBF0FBEB1
:103910002DBF4CCF80911D038F7B80931D03809121
:10392000E1019091E20100D000D02BE43FE0ADB77F
:10393000BEB712963C932E93119714969C938E9338
:1039400013970E940B4E0F900F900F900F9020CF67
:103950000E94FB1AE0901003F090110300911203F3
:103960001091130320916101309162014091630134
:10397000509164016091FC027091FD028091FE0201
:103980009091FF0269877A878B879C87A0900C03B0
:10399000B0900D03C0900E03D0900F03809198015A
:1039A000909199019E878D876090480170904901A0
:1039B00080904A0190904B019091DC019983209076
:1039C0002E0230902F0240903002509031026091D0
:1039D00090027091910280919202909193026D8376
:1039E0007E838F8398878DB79EB786970FB6F8949E
:1039F0009EBF0FBE8DBFEDB7FEB731966AE570E191
:103A0000ADB7BEB712967C936E931197E282F382A4
:103A100004831583268337834087518729853A8518
:103A20004B855C852287338744875587A686B78672
:103A3000C08AD18A4D855E85538B428B648A758A94
:103A4000868A978A8091DF019091E001918F808F23
:103A50008091860190918701938F828F5981548F35
:103A6000158E268E378E40A251A26D817E818F8168
:103A7000988562A373A384A395A30E940B4E8DB770
:103A80009EB786960FB6F8949EBF0FBE8DBF3ACEF6
:103A90000E94FB1AE0901003F090110300911203B2
:103AA0001091130320912E0230912F024091300289
:103AB00050913102A0909002B0909102C090920279
:103AC000D090930280918C0190918D01ADB7BEB7DB
:103AD00050970FB6F894BEBF0FBEADBFEDB7FEB79F
:103AE00031966FE370E112967C936E931197E282A8
:103AF000F382048315832683378340875187A28608
:103B0000B386C486D586978786870E940B4EEDB70D
:103B1000FEB770960FB6F894FEBF0FBEEDBF01CE94
:103B20000E94FB1A2091100330911103409112035F
:103B300050911303E0906101F090620100916301E4
:103B4000109164016090FC027090FD028090FE0272
:103B50009090FF0220900C0330900D0340900E03D4
:103B600050900F0360919801709199017E836D834D
:103B700080918C0290918D02A0918E02B0918F0263
:103B800089839A83AB83BC8360918C0270918D0290
:103B900080918E0290918F02A0900803B09009034B
:103BA000C0900A03D0900B03ADB7BEB75E970FB6B7
:103BB000F894BEBF0FBEADBFEDB7FEB73196FA8722
:103BC000E987E9E0F0E11296FC93EE931197E9851D
:103BD000FA852283338344835583A985BA85169653
:103BE000ED92FD920D931C931997E985FA856286F3
:103BF000738684869586A985BA851E962D923D92F8
:103C00004D925C925197ED81FE815396FC93EE9319
:103C1000529729813A814B815C81A985BA85549656
:103C20002D933D934D935C93579720918A0158961D
:103C30002C93589759961C92A60195010E947D4895
:103C4000E985FA85628F738F848F958F0E940B4E62
:103C50002DB73EB7225E3F4F0FB6F8943EBF0FBE62
:103C60002DBF6ECD0E94FB1A40913A0250913B024B
:103C70002091C3023091C40280911E0390911F03D2
:103C8000A0912003B09121036DB77EB76A507040B8
:103C90000FB6F8947EBF0FBE6DBFEDB6FEB60894AA
:103CA000E11CF11C67ED7FE0EDB7FEB77283618325
:103CB000F701538342833583248386839783A087C8
:103CC000B1870E940B4E80911D03877F80931D0357
:103CD0002DB73EB7265F3F4F0FB6F8943EBF0FBEDD
:103CE0002DBF38CD0E94FB1A40913A0250913B0201
:103CF0002091C3023091C40280911E0390911F0352
:103D0000A0912003B09121036DB77EB76A50704037
:103D10000FB6F8947EBF0FBE6DBFEDB6FEB6089429
:103D2000E11CF11C60EA7FE0EDB7FEB772836183AE
:103D3000F701538342833583248386839783A08747
:103D4000B1870E940B4E80911D038F7E80931D03CF
:103D50002DB73EB7265F3F4F0FB6F8943EBF0FBE5C
:103D60002DBF02CD80911D038F7D80931D03209177
:103D7000E1013091E2018091E3019091E40100D0F2
:103D800000D000D0EDB7FEB731964EE65FE0ADB79C
:103D9000BEB712965C934E9311973383228395831B
:103DA00084830E940B4EEDB7FEB736960FB6F8949B
:103DB000FEBF0FBEEDBFE2CC0E9437168091ED0131
:103DC0009091EE0101969093EE018093ED018F7337
:103DD0009070009709F491C06091FC027091FD020F
:103DE0008091FE029091FF02209110033091110307
:103DF00040911203509113030E94314A181634F473
:103E000082E090E090938901809388016091FC02A8
:103E10007091FD028091FE029091FF0220911003AB
:103E20003091110340911203509113030E94E24814
:103E300087FF09C08091ED019091EE018F7790701E
:103E4000009709F453C060911003709111038091A1
:103E500012039091130323E333E347E451E40E94F8
:103E6000314A87FD09C08091ED019091EE018F7775
:103E70009070009709F444C0609110037091110391
:103E800080911203909113032DEC3CEC44E451E437
:103E90000E94314A87FD08C08091ED019091EE01AA
:103EA0008F7790700097B1F16091100370911103BA
:103EB000809112039091130323EC35EF40E451E419
:103EC0000E94314A87FD08C08091ED019091EE017A
:103ED0008F779070009759F18091D2019091D30122
:103EE00087FF089581E00E94E711089581E090E046
:103EF0009093890180938801A6CF0E9495136CCF7F
:103F000083E00E94E7118091D2019091D30187FF55
:103F1000E8CFE8CF83E00E94E71182E00E94E7113A
:103F20008091D2019091D30187FFDBCFDBCF82E07C
:103F30000E94E7118091D2019091D30187FFD1CFE8
:103F4000D1CF80911D0380FD32C078948091D4013F
:103F50009091D5010097E9F08091A0019091A10185
:103F6000A091A201B091A3010097A105B10589F428
:103F70008091940190919501A0919601B091970143
:103F80000097A105B10529F483B7817F866083BFBF
:103F900003C083B7817F83BFF89483B7816083BFF9
:103FA0007894889583B78E7F83BF789408958091A5
:103FB0001D038E7F80931D030E94DC1EC6CF0F93CE
:103FC0001F93CF93DF9310E00E945F438823A1F1FA
:103FD0008091AD039091AE030E949D4DEC018FEF57
:103FE000CF3FD80789F3CD30C9F0C231D10509F4EC
:103FF00044C0CF37D10519F1C830D10501F1609126
:10400000AF037091B003CE010E94DF4DE12FF0E0CD
:10401000E653FD4FC0831F5F1133B0F2212F30E014
:10402000F901E653FD4F10822F5F3F4FC901DF9129
:10403000CF911F910F9108950E94A11FC5CF112309
:1040400011F410E0C1CF6091AF037091B00388E02C
:1040500090E00E94DF4D6091AF037091B00380E269
:1040600090E00E94DF4D6091AF037091B00388E053
:1040700090E00E94DF4D1150CFCF6091AF0370915F
:10408000B0038DE090E00E94DF4D1123D1F2CAEC25
:10409000D2E000E06091AF037091B003899190E0AD
:1040A0000E94DF4D0F5F0117A8F3B6CFEF92FF928A
:1040B0000F931F93CF93DF9300D08FE091E1EDB783
:1040C000FEB7928381830E940B4E0F900F908091D8
:1040D000AD039091AE030E94DF1F8230910534F052
:1040E0008091CA02893749F0893539F0DF91CF9143
:1040F0001F910F91FF90EF90089500D0C1E7D1E19B
:10410000EDB7FEB7D283C1830E940B4E85E091E1EB
:10411000EDB7FEB7928381830E940B4EEDB7FEB7D9
:10412000D283C1830E940B4E8FEF8093B80280939D
:10413000B9028093BA028093BB028093BC02809341
:10414000BD028093BE028093BF020F900F9088EB58
:1041500092E064E470E049E050E00E94D04E10929A
:10416000D90189ED91E065E370E041E050E00E9403
:10417000D04E11E010938A018AE891E062E470E089
:1041800041E050E00E94D04E10938B018BE891E00B
:1041900063E470E041E050E00E94D04E0F2EFEEA52
:1041A000EF2EF7E4FF2EF1EE0F2FFCE31F2FF02D83
:1041B000E0924C01F0924D0100934E0110934F019B
:1041C0008CE491E060E070E044E050E00E94D04E6A
:1041D000E0925001F092510100935201109353016B
:1041E00080E591E064E070E044E050E00E94D04E51
:1041F000E0925401F092550100935601109357013B
:1042000084E591E068E070E044E050E00E94D04E28
:104210000F2EFAE0EF2EF7EDFF2EF3EA0F2FFBE360
:104220001F2FF02DE0925801F092590100935A018E
:1042300010935B0188E591E06CE070E044E050E0B1
:104240000E94D04EE0925C01F0925D0100935E010D
:1042500010935F018CE591E060E170E044E050E094
:104260000E94D04E0F2EF0E0EF2EF0E0FF2EF0E097
:104270000F2FF0E01F2FF02DE092C501F092C60144
:104280000093C7011093C80185EC91E064E170E0F0
:1042900044E050E00E94D04EE092C901F092CA0181
:1042A0000093CB011093CC0189EC91E068E170E0C0
:1042B00044E050E00E94D04E83E393E3A3E2B1E4F4
:1042C0008093610190936201A0936301B0936401B4
:1042D00081E691E06DE170E044E050E00E94D04E54
:1042E0000F2EF0E0EF2EF0E0FF2EF8E50F2FF1E4B7
:1042F0001F2FF02DE0926901F0926A0100936B018B
:1043000010936C0189E691E065E270E044E050E0D2
:104310000E94D04E86E696E6A6E6B1E480936D0153
:1043200090936E01A0936F01B09370018DE691E0C0
:1043300069E270E044E050E00E94D04E80E090E0FE
:10434000AAE7B5E48093820190938301A09384014E
:10435000B093850182E891E06EE370E044E050E0C4
:104360000E94D04E80E090E0A0E9B1E48093650126
:1043700090936601A0936701B093680185E691E090
:1043800061E270E044E050E00E94D04EE0926101B2
:10439000F092620100936301109364010F2EF0E02C
:1043A000EF2EF0E0FF2EF0EA0F2FF0E41F2FF02D9C
:1043B000E0927101F0927201009373011093740105
:1043C00081E791E06DE270E044E050E00E94D04E61
:1043D000E0927501F09276010093770110937801D5
:1043E00085E791E061E370E044E050E00E94D04E48
:1043F00080E090E0A0E4B1E48093790190937A01A9
:10440000A0937B01B0937C0189E791E066E370E0C3
:1044100044E050E00E94D04E8DEC9CECACE4BFE355
:1044200080937D0190937E01A0937F01B0938001E2
:104430008DE791E06AE370E044E050E00E94D04EE6
:1044400085E08093600180E691E06CE170E041E0FE
:1044500050E00E94D04EDF91CF911F910F91FF90BD
:10446000EF9008950E94FB1A00D081E791E1EDB72B
:10447000FEB7928381830E940B4E0F900F90089598
:1044800080E09FE00E94294385EC9EE00E94294342
:104490008091A601882389F183E191E000D000D0CA
:1044A0002DEB3EE0EDB7FEB7328321839483838307
:1044B0000E940B4E8091B9030F900F900F900F90B8
:1044C00083FD1EC088E291E000D000D022EB3EE0E8
:1044D000EDB7FEB732832183948383830E940B4E12
:1044E0000F900F9081E791E1EDB7FEB79283818342
:1044F0000E940B4E0F900F90089588E191E0CECF6F
:104500008FE191E0E1CF8CEA9EE00E94294308957B
:10451000EF92FF920F931F93CF93DF930E9440225D
:1045200000D086EA9EE0ADB7BEB712969C938E93FC
:1045300011970E940B4E0F900F900E94322200D0D4
:104540008EE99EE0CDB7DEB79A8389830E940B4E39
:104550000F900F9060919402709195028091960255
:10456000909197020E94C50900D084E99EE0EDB7C2
:10457000FEB7928381830E940B4E0F900F90609143
:1045800026027091270280912802909129020E94B0
:10459000C5098091D901882309F4DFC280911003F5
:1045A00090911103A0911203B091130300D000D099
:1045B00000D02EE73EE0CDB7DEB73A832983EDB7D2
:1045C000FEB783839483A583B6830E940B4E2DB7D9
:1045D0003EB72A5F3F4F0FB6F8943EBF0FBE2DBFC8
:1045E0008091FC029091FD02A091FE02B091FF0229
:1045F00000D000D000D023E53EE0CDB7DEB73A834F
:104600002983EDB7FEB783839483A583B6830E9485
:104610000B4E8CE39EE0ADB7BEB712969C938E9383
:10462000119780916D0190916E01A0916F01B091F1
:104630007001CDB7DEB78B839C83AD83BE830E94B0
:104640000B4E85E29EE0EDB7FEB7928381838091A9
:10465000690190916A01A0916B01B0916C01CDB795
:10466000DEB78B839C83AD83BE830E940B4E80910B
:10467000610190916201A0916301B09164012FE00A
:104680003EE0EDB7FEB732832183CDB7DEB78B8333
:104690009C83AD83BE830E940B4E80912E0290912D
:1046A0002F02A0913002B091310228EF3DE0EDB72A
:1046B000FEB732832183CDB7DEB78B839C83AD8376
:1046C000BE830E940B4E80910C0390910D03A0912C
:1046D0000E03B0910F0323EE3DE0EDB7FEB732833A
:1046E0002183CDB7DEB78B839C83AD83BE830E94CD
:1046F0000B4E8091900290919102A0919202B09104
:1047000093022CEC3DE0EDB7FEB732832183CDB7A9
:10471000DEB78B839C83AD83BE830E940B4E80EB00
:104720009DE0EDB7FEB792838183809171019091F6
:104730007201A0917301B0917401CDB7DEB78B8384
:104740009C83AD83BE830E940B4E85E99DE0EDB74F
:10475000FEB7928381838091750190917601A0913B
:104760007701B0917801CDB7DEB78B839C83AD83A1
:10477000BE830E940B4E0F900F900F900F9088E811
:104780009DE0EDB7FEB7928381830E940B4E0F90A0
:104790000F9060911E0270911F02809120029091F3
:1047A00021020E94C50900D000D000D086E69DE01D
:1047B000ADB7BEB712969C938E93119780917901F5
:1047C00090917A01A0917B01B0917C01CDB7DEB7C9
:1047D0008B839C83AD83BE830E940B4E8091DC0152
:1047E000EDB7FEB736960FB6F894FEBF0FBEEDBF1D
:1047F000882309F0D8C18091DD01882309F0C7C161
:1048000000D08DE09DE0EDB7FEB7928381830E94DA
:104810000B4E0F900F900E940A1200D0C1E7D1E119
:10482000ADB7BEB71296DC93CE9311970E940B4E94
:104830000F900F908091DE01882309F09CC100D079
:1048400000D000D085EC9CE0ADB7BEB712969C932B
:104850008E93119780917D0190917E01A0917F01AF
:10486000B0918001EDB7FEB783839483A583B683AF
:104870000E940B4E2DB73EB72A5F3F4F0FB6F894FC
:104880003EBF0FBE2DBF8091D601882309F4AFC073
:104890008091480190914901A0914A01B0914B014A
:1048A00000D000D000D02FEA3CE0EDB7FEB7328355
:1048B000218383839483A583B6830E940B4E2DB7F7
:1048C0003EB72A5F3F4F0FB6F8943EBF0FBE2DBFD5
:1048D0008091B8028F3F09F474C100D0EDB7FEB7E4
:1048E000D283C1830E940B4E0F900F9080918A015A
:1048F000882309F0B4C000D000D000D083EB9BE047
:10490000CDB7DEB79A838983809165019091660166
:10491000A0916701B0916801EDB7FEB783839483DE
:10492000A583B6830E940B4E6091FF017091000237
:10493000809101029091020220E030E0A9010E94E2
:104940007E4820910302309104024091050250916B
:1049500006020E947E482091070230910802409191
:10496000090250910A020E947E4820910B02309168
:104970000C0240910D0250910E020E947E487B0174
:104980008C0120910F023091100240911102509140
:104990001202CDB7DEB72196E4E9FBE0ADB7BEB7B2
:1049A0001296FC93EE931197CA01B9012E2D3F2D5B
:1049B000402F512F0E947E4820E030E040EA50E432
:1049C0000E94E6486A837B838C839D830E940B4E02
:1049D000CDB7DEB726960FB6F894DEBF0FBECDBFBB
:1049E000DF91CF911F910F91FF90EF90089500D02C
:1049F00000D0EDB7FEB7319685E69CE0ADB7BEB707
:104A000012969C938E9311978091D7018283138283
:104A10000E940B4E8091480190914901A0914A015A
:104A2000B0914B0100D024E43CE0CDB7DEB73A832F
:104A30002983EDB7FEB783839483A583B6830E9451
:104A40000B4E2DB73EB72A5F3F4F0FB6F8943EBFCF
:104A50000FBE2DBF80918A01882309F44CCF20918D
:104A6000E5013091E6014091E7015091E801809124
:104A7000E9019091EA01A091EB01B091EC016DB7D1
:104A80007EB76A5070400FB6F8947EBF0FBE6DBF00
:104A9000EDB7FEB7319669E27CE0CDB7DEB77A8339
:104AA0006983228333834483558386839783A087D6
:104AB000B1870E940B4E20918B01EDB7FEB73A965D
:104AC0000FB6F894FEBF0FBEEDBF222309F0AAC0B7
:104AD00040913A0250913B022091C3023091C402AE
:104AE00080911E0390911F03A0912003B091210398
:104AF000CDB7DEB72A970FB6F894DEBF0FBECDBF95
:104B0000EDB7FEB731966AEE7BE07A836983538313
:104B100042833583248386839783A087B1870E944D
:104B20000B4E20916001EDB7FEB736960FB6F894A4
:104B3000FEBF0FBEEDBF31968EEC9BE0ADB7BEB7AA
:104B400012969C938E931197228313820E940B4E90
:104B50000F900F900F900F90CECE809110039091F8
:104B60001103A0911203B091130300D000D000D024
:104B700028E63EE020CD00D08DEE9CE0EDB7FEB7FC
:104B8000928381830E940B4E0F900F9058CE00D0DD
:104B900085E29DE0CDB7DEB79A8389830E940B4EF4
:104BA0000F900F902DCE00D084E49DE0ADB7BEB73E
:104BB00012969C938E9311970E940B4E0F900F901C
:104BC0001ACE8091B9028F3F09F087CE8091BA0248
:104BD0008F3F09F082CE8091BB028F3F09F07DCEDE
:104BE0008091BC028F3F09F078CE8091BD028F3F4B
:104BF00009F073CE8091BE028F3F09F06ECE809196
:104C0000BF028F3F09F069CE00D08EE79CE0ADB7C0
:104C1000BEB712969C938E9311970E940B4E0F90E5
:104C20000F905BCE00D000D0EDB7FEB7319689E192
:104C30009CE0ADB7BEB712969C938E9311972283DA
:104C400013820E940B4E0F900F900F900F9040CF49
:104C5000EF92FF920F931F93CF93DF9380911003F6
:104C600090911103A0911203B091130300D000D0D2
:104C700000D02BE63BE0EDB7FEB732832183838380
:104C80009483A583B6830E940B4E8DB79EB706967C
:104C90000FB6F8949EBF0FBE8DBF8091AD0390916B
:104CA000AE030E94DF1F823050F18AEC92E00E9436
:104CB000324CE0901003F090110300911203109118
:104CC00013032091500130915101409152015091B4
:104CD00053010E94354AA80197010E94E64860935B
:104CE000500170935101809352019093530180E5DC
:104CF00091E064E070E044E050E00E94D04E00D0CB
:104D0000C1E7D1E1EDB7FEB7D283C1830E940B4E5C
:104D10008091FC029091FD02A091FE02B091FF02F1
:104D200000D000D024E43BE0EDB7FEB7328321830E
:104D300083839483A583B6830E940B4E8DB79EB761
:104D400006960FB6F8949EBF0FBE8DBF8091AD033F
:104D50009091AE030E94DF1F823050F18AEC92E006
:104D60000E94324CE090FC02F090FD020091FE02A5
:104D70001091FF0220914C0130914D0140914E0164
:104D800050914F010E94354AA80197010E94E648C0
:104D900060934C0170934D0180934E0190934F01AD
:104DA0008CE491E060E070E044E050E00E94D04E7E
:104DB00000D0EDB7FEB7D283C1830E940B4E809125
:104DC0002E0290912F02A0913002B091310200D0BA
:104DD00000D02EE13BE0EDB7FEB732832183838321
:104DE0009483A583B6830E940B4E8DB79EB706961B
:104DF0000FB6F8949EBF0FBE8DBF8091AD0390910A
:104E0000AE030E94DF1F823050F18AEC92E00E94D4
:104E1000324CE0902E02F0902F020091300210915F
:104E20003102209154013091550140915601509129
:104E300057010E94354AA80197010E94E6486093F5
:104E4000540170935501809356019093570184E566
:104E500091E068E070E044E050E00E94D04E00D065
:104E6000EDB7FEB7D283C1830E940B4E80919002B2
:104E700090919102A0919202B091930200D000D043
:104E800028EF3AE0EDB7FEB7328321838383948322
:104E9000A583B6830E940B4E8DB79EB706960FB6BC
:104EA000F8949EBF0FBE8DBF8091AD039091AE036D
:104EB0000E94DF1F823060F18AEC92E00E94324C47
:104EC0009B01AC01609190027091910280919202DD
:104ED000909193020E947D489B01AC016091C501B5
:104EE0007091C6018091C7019091C8010E947E48CF
:104EF0006093C5017093C6018093C7019093C80168
:104F000085EC91E064E170E044E050E00E94D04E16
:104F100000D0EDB7FEB7D283C1830E940B4E8091C3
:104F20000C0390910D03A0910E03B0910F0300D0DC
:104F300000D024ED3AE0EDB7FEB7328321838383BE
:104F40009483A583B6830E940B4E8DB79EB70696B9
:104F50000FB6F8949EBF0FBE8DBF8091AD039091A8
:104F6000AE030E94DF1F823060F18AEC92E00E9463
:104F7000324C9B01AC0160910C0370910D03809148
:104F80000E0390910F030E947D489B01AC0160913C
:104F9000C9017091CA018091CB019091CC010E940E
:104FA0007E486093C9017093CA018093CB019093AE
:104FB000CC0189EC91E068E170E044E050E00E94AF
:104FC000D04E00D0EDB7FEB7D283C1830E940B4E06
:104FD0000F900F90DF91CF911F910F91FF90EF9065
:104FE0000895CF93DF9300D000D000D08BEA9AE0F1
:104FF000EDB7FEB7928381838091690190916A0138
:10500000A0916B01B0916C0183839483A583B683D7
:105010000E940B4E8DB79EB706960FB6F8949EBFB2
:105020000FBE8DBF8091AD039091AE030E94DF1F34
:105030008230A0F08AEC92E00E94324C60936901C9
:1050400070936A0180936B0190936C0189E691E003
:1050500065E270E044E050E00E94D04E00D0C1E72D
:10506000D1E1EDB7FEB7D283C1830E940B4E00D0D1
:1050700000D082E89AE0EDB7FEB7928381838091F9
:105080006D0190916E01A0916F01B09170018383C9
:105090009483A583B6830E940B4E8DB79EB7069668
:1050A0000FB6F8949EBF0FBE8DBF8091AD03909157
:1050B000AE030E94DF1F8230A0F08AEC92E00E94D3
:1050C000324C60936D0170936E0180936F019093E9
:1050D00070018DE691E069E270E044E050E00E94EA
:1050E000D04E00D0EDB7FEB7D283C1830E940B4EE5
:1050F0008091690190916A01A0916B01B0916C015E
:105100008093610190936201A0936301B093640165
:105110000F900F90DF91CF91089585E79AE00E945C
:10512000294387E69AE00E9429438BE49AE00E9493
:10513000294380E39AE00E9429438DE09AE00E948F
:10514000294381EF99E00E9429438BEC99E00E946A
:1051500029438CEA99E00E94294389E899E00E945A
:10516000294384E799E00E94294388E599E00E9459
:1051700029438EE399E00E94294383E299E00E944B
:1051800029438EEF98E00E94294384EE98E00E9424
:105190002943089500D087ED98E0EDB7FEB79283DC
:1051A00081830E940B4E8091A4010F900F90882361
:1051B00009F408950E94094308958AEC98E00E943A
:1051C000294382EB98E00E9429438BE998E00E94F2
:1051D00029438DE898E00E9429438BE798E00E94DC
:1051E000294386E698E00E9429438BE498E00E94D8
:1051F00029438AE398E00E9429438BE298E00E94C9
:1052000029438BE198E00E9429438DEF97E00E94AB
:1052100029438CED97E00E9429438DEB97E00E9493
:1052200029438BE997E00E9429438091C40182FFC2
:1052300017C08091C301882309F491C082E391E0F3
:1052400000D000D029E837E0EDB7FEB732832183E4
:10525000948383830E940B4E0F900F900F900F90BA
:1052600080918A01882309F071C08FE291E000D01B
:1052700000D026E737E0EDB7FEB732832183948371
:1052800083830E940B4E0F900F900F900F90809190
:105290008B01882309F057C08FE291E000D000D045
:1052A0002BE537E0EDB7FEB7328321839483838308
:1052B0000E940B4E0F900F908DE397E0EDB7FEB775
:1052C000928381830E940B4E0F900F9089E297E0AA
:1052D0000E94294388E097E00E9429438091C401FD
:1052E00080FF18C0809146018823B1F182E391E0EC
:1052F00000D000D022EF36E0EDB7FEB73283218335
:10530000948383830E940B4E8091C4010F900F9071
:105310000F900F9081FF16C0809147018823C9F03C
:1053200082E391E000D000D025ED36E0EDB7FEB786
:1053300032832183948383830E940B4E0F900F90BE
:105340000F900F90089582E391E0A8CF82E391E05F
:105350008ECF8FE291E0E6CF8FE291E0C9CF8FE26E
:1053600091E06ECF2F923F924F925F926F927F9219
:105370008F929F92AF92BF92CF92DF92EF92FF9265
:105380000F931F93CF93DF93822E732E642E552E8F
:10539000462E372E282E992E263609F48EC0282D1B
:1053A000372D462D552D642D732D822D992D06E612
:1053B000A02E16E6B12ECC24DD24EE24FF2400E03E
:1053C00010E00E948B448230E0F1882D893609F488
:1053D000ADC3282D372D462D552D642D732D822DCF
:1053E000992DF9E6AF2EE4E7BE2ECC24DD24EE2481
:1053F000FF2400E010E00E948B44823008F0F1C0EE
:10540000E82DE83609F4D8C1882D853609F49BC10A
:10541000E82DE63709F44AC10E94CA28DF91CF91EE
:105420001F910F91FF90EF90DF90CF90BF90AF90C2
:105430009F908F907F906F905F904F903F902F90B4
:105440000895882D8C3609F4DCC3282D372D462D80
:10545000552D642D732D822D992DBCE6AB2EA1E622
:10546000BA2ECC24DD24EE24FF2400E010E00E94BC
:105470008B44823008F08BC0E82DED3609F406C26B
:10548000F82DF93609F4F9C2982D983629F67720C7
:1054900019F6662009F6552009F0BECF442009F020
:1054A000BBCF332009F0B8CF222009F0B5CF992027
:1054B00009F0B2CF0E948D28B1CF363609F06FCFF8
:1054C000442309F06CCF552309F069CF662309F016
:1054D00066CF772309F063CF882309F060CF992343
:1054E00009F05DCF8091A501882309F495CF00D004
:1054F0008BE596E0EDB7FEB7928381830E940B4E59
:1055000000D000D08DE396E0EDB7FEB792838183A3
:105510008091820190918301A0918401B0918501D5
:1055200083839483A583B6830E940B4E8DB79EB769
:1055300006960FB6F8949EBF0FBE8DBF8091AD0347
:105540009091AE030E94DF1F82309105A4F08AEC97
:1055500092E00E94324C60938201709383018093A9
:1055600084019093850182E891E06EE370E044E06D
:1055700050E00E94D04E00D081E791E1EDB7FEB738
:10558000928381830E940B4E0F900F9047CFE82D9E
:10559000E13609F454C2882D863709F4F7C1E82DA5
:1055A000E13609F039CFF72DF23609F035CF662014
:1055B00009F032CF552009F02FCF442009F02CCF2D
:1055C000332009F029CF222009F026CF992009F0B5
:1055D00023CF8091A501882309F41ECF0E94F127D3
:1055E0001DCF882D8C3609F478C1E82DE03709F4F9
:1055F00067C1E82DE73609F00FCFF72DF63709F030
:105600000BCF662009F008CF552009F005CF4420C4
:1056100009F002CF332009F0FFCE222009F0FCCEA2
:10562000992009F0F9CE8091A501882309F4F4CEE0
:105630008091610190916201A0916301B091640138
:1056400000D000D000D023E236E0EDB7FEB73283C1
:10565000218383839483A583B6830E940B4E8DB7E9
:105660009EB706960FB6F8949EBF0FBE8DBF809171
:10567000AD039091AE030E94DF1F823091050CF4C0
:105680007ACF8AEC92E00E94324C60936101709371
:105690006201809363019093640181E691E06DE182
:1056A00070E044E050E00E94D04E65CFF72DF63612
:1056B00009F0B2CE662009F0AFCE552009F0ACCE8D
:1056C000442009F0A9CE332009F0A6CE222009F00B
:1056D000A3CE992009F0A0CE81E09091D90191113B
:1056E00080E08093D901882309F4E4C286E391E045
:1056F00000D000D025EB36E0EDB7FEB73283218332
:10570000948383830E940B4E0F900F900F900F9005
:105710008091D901882309F0D0C289ED91E065E339
:1057200070E041E050E00E94D04E8091D901882382
:1057300009F474CE81E691E06DE170E044E050E060
:105740000E94C04E6BCE972D943709F065CE66202F
:1057500009F062CE552009F05FCE442009F05CCEFE
:10576000332009F059CE222009F056CE992009F0B5
:1057700053CE8091A501882309F44ECE0E94951343
:105780008091480190914901A0914A01B0914B014B
:1057900000D000D000D02BE635E0EDB7FEB7328365
:1057A000218383839483A583B6830E940B4E0F903D
:1057B0000F900F900F90E0CEF72DF23709F02CCE1E
:1057C000662009F029CE552009F026CE442009F0A4
:1057D00023CE332009F020CE222009F01DCE9920BF
:1057E00009F01ACE8091A501882309F415CE00D0C6
:1057F00000D000D080E895E0EDB7FEB792838183BA
:1058000080917D0190917E01A0917F01B0918001F6
:1058100083839483A583B6830E940B4E8DB79EB776
:1058200006960FB6F8949EBF0FBE8DBF8091AD0354
:105830009091AE030E94DF1F823091050CF49BCE45
:1058400060917D0170917E0180917F019091800136
:105850002DEC3CEC4CEC5DE30E94314A18160CF048
:105860008ACE8AEC92E00E94324C60937D01709364
:105870007E0180937F01909380018DE791E06AE340
:1058800070E044E050E00E94D04E75CE772009F0E1
:10589000C3CD662009F0C0CD552009F0BDCD442010
:1058A00009F0BACD332009F0B7CD222009F0B4CDEC
:1058B000992009F0B1CD1092D8010E94DD28AECD1B
:1058C000F72DFC3609F0A8CD862D853609F0A4CD3C
:1058D000952D983609F0A0CDE1CD972D963709F09A
:1058E0009BCD662009F098CD552009F095CD442038
:1058F00009F092CD332009F08FCD222009F08CCD14
:10590000992009F089CD8091A501882309F484CDDF
:1059100000D000D000D084E096E0EDB7FEB79283CF
:1059200081838091650190916601A0916701B0919A
:10593000680183839483A583B6830E940B4E8DB741
:105940009EB706960FB6F8949EBF0FBE8DBF80918E
:10595000AD039091AE030E94DF1F823091050CF4DD
:105960000ACE8AEC92E00E94324C609365017093FB
:105970006601809367019093680185E691E061E29A
:1059800070E044E050E00E94D04EF5CD972D943663
:1059900009F042CD662009F03FCD552009F03CCDFD
:1059A000442009F039CD332009F036CD222009F00A
:1059B00033CD992009F030CD8091A501882309F4D9
:1059C0002BCD00D000D000D08EE995E0EDB7FEB72A
:1059D000928381838091790190917A01A0917B01DA
:1059E000B0917C0183839483A583B6830E940B4E80
:1059F0008DB79EB706960FB6F8949EBF0FBE8DBFAB
:105A00008091AD039091AE030E94DF1F823091051B
:105A10000CF4B1CD8AEC92E00E94324C6093790193
:105A200070937A0180937B0190937C0189E791E0E8
:105A300066E370E044E050E00E94D04E9CCDF72D2C
:105A4000F33609F0B0CD662009F0E6CC552009F018
:105A5000E3CC442009F0E0CC332009F0DDCC222057
:105A600009F0DACC992009F0D7CC8091A5018823E0
:105A700009F4D2CC0E942826D1CC872D813609F09A
:105A8000CBCC662009F0C8CC552009F0C5CC442009
:105A900009F0C2CC332009F0BFCC222009F0BCCCE5
:105AA000992009F0B9CC8091A501882309F4B4CCE0
:105AB00000D000D000D08DED95E0EDB7FEB7928319
:105AC00081838091710190917201A0917301B091D5
:105AD000740183839483A583B6830E940B4E8DB794
:105AE0009EB706960FB6F8949EBF0FBE8DBF8091ED
:105AF000AD039091AE030E94DF1F823091050CF43C
:105B00003ACD8AEC92E00E94324C6093710170931E
:105B10007201809373019093740181E791E06DE2CB
:105B200070E044E050E00E94D04E25CD972D943790
:105B300009F04FCC662009F04CCC552009F049CC37
:105B4000442009F046CC332009F043CC222009F050
:105B500040CC992009F03DCC8091A501882309F41F
:105B60005BCC0E94440B00D0C1E7D1E1EDB7FEB79A
:105B7000D283C1830E940B4E8BE495E0EDB7FEB754
:105B8000928381830E940B4E0F900F908091AD0302
:105B90009091AE030E94DF1F823091053CF08AECA9
:105BA00092E00E94364C883008F4AFC000D0EDB7C8
:105BB000FEB7D283C1830E940B4E8AE295E0EDB717
:105BC000FEB7928381830E940B4E0F900F908091BD
:105BD000AD039091AE030E94DF1F823091053CF02F
:105BE0008AEC92E00E94364C883008F472C000D0F3
:105BF000EDB7FEB7D283C1830E940B4E0F900F907A
:105C00000DCC972D913609F020CC662009F01DCCE3
:105C1000552009F01ACC442009F017CC332009F0A4
:105C200014CC222009F011CC992009F00ECC8091DF
:105C3000A501882309F4F0CB00D000D000D087EB79
:105C400095E0EDB7FEB792838183809175019091C5
:105C50007601A0917701B091780183839483A58325
:105C6000B6830E940B4E8DB79EB706960FB6F8947A
:105C70009EBF0FBE8DBF8091AD039091AE030E9479
:105C8000DF1F823091050CF476CC8AEC92E00E9402
:105C9000324C6093750170937601809377019093F5
:105CA000780185E791E061E370E044E050E00E9414
:105CB000D04E61CC89E391E01BCD00D084E996E021
:105CC000EDB7FEB7928381830E940B4E0F900F9029
:105CD00024CD90E0FC01EE0FFF1FEE0FFF1FEE0F33
:105CE000FF1FE80FF91FA4E1B3E0E45CFD4F89E07A
:105CF00001900D928150E1F784E193E06DE470E052
:105D000049E050E00E94D04E72CF90E0FC01EE0FCF
:105D1000FF1FEE0FFF1FEE0FFF1FE80FF91FA8EB8D
:105D2000B2E0E45CFD4F89E001900D928150E1F713
:105D300088EB92E064E470E049E050E00E94D04ECD
:105D400035CF2F923F924F925F926F927F928F92B8
:105D50009F92AF92BF92CF92DF92EF92FF920F93FA
:105D60001F93DF93CF93CDB7DEB72C970FB6F89480
:105D7000DEBF0FBECDBF822E732E642E552E462E53
:105D8000372E282E992E233709F446C1282D372D7A
:105D9000462D552D642D732D822D992D03E7A02EB0
:105DA00013E7B12ECC24DD24EE24FF2400E010E024
:105DB0000E948B44823008F4D4C0282D213309F48A
:105DC0007FC5282D372D462D552D642D732D822D01
:105DD000992DB1E3AB2EA1E3BA2EF1E7CF2EDD244E
:105DE000EE24FF2400E010E00E948B44823008F093
:105DF00032C1782D723709F408C5282D372D462D6C
:105E0000552D642D732D822D992DE2E7AE2E02E7DC
:105E1000B02E15E6C12EDD24EE24FF2400E010E0B4
:105E20000E948B44823008F408C2F82DF53709F43B
:105E3000A8C6682D603309F033C1772D713309F09E
:105E40002FC1862D813709F02BC1552009F028C1BB
:105E5000442009F025C1332009F022C1222009F095
:105E60001FC1992009F01CC100D08DE593E0ADB7AA
:105E7000BEB712969C938E9311970E940B4EEDB76E
:105E8000FEB77C970FB6F894FEBF0FBEEDBF3196FC
:105E90008BE293E0ADB7BEB712969C938E931197A9
:105EA0008091980290919902A0919A02B0919B02E0
:105EB00082839383A483B58380919C0290919D02F9
:105EC000A0919E02B0919F0286839783A087B1879D
:105ED0008091A0029091A102A091A202B091A30290
:105EE00082879387A487B5878091A4029091A502A9
:105EF000A091A602B091A70286879787A08BB18B4D
:105F00008091A8029091A902A091AA02B091AB023F
:105F1000828B938BA48BB58B8091B0029091B10250
:105F2000A091B202B091B302868B978BA08FB18FF4
:105F30008091AC029091AD02A091AE02B091AF02FF
:105F4000828F938FA48FB58F0E940B4EEDB7FEB753
:105F50007E960FB6F894FEBF0FBEEDBF21E030E095
:105F6000A1C0282D203309F485C4282D372D462DB6
:105F7000552D642D732D822D992DB0E3AB2EA1E705
:105F8000BA2ECC24DD24EE24FF2400E010E00E9491
:105F90008B44823008F0A0C0682D603709F4F0C34C
:105FA000282D372D462D552D642D732D822D992D9D
:105FB000F0E7AF2EECE6BE2ECC24DD24EE24FF2449
:105FC00000E010E00E948B44823008F4B8C1A82D94
:105FD000A93609F424C6E82DE73709F061C0F72D8A
:105FE000FF3609F05DC0662009F05AC0552009F05F
:105FF00057C0442009F054C0332009F051C022207A
:1060000009F04EC0992009F04BC00E94440B8091CA
:10601000A4018823E9F04FC4333709F0B7CE4423F5
:1060200009F0B4CE552309F0B1CE662309F0AECE07
:10603000772309F0ABCE882309F0A8CE992309F085
:10604000A5CE0E9488228091A401882309F033C440
:1060500021E030E027C0982D943709F4EEC3282DB5
:10606000372D462D552D642D732D822D992DB4E796
:10607000AB2EAFE6BA2EFFE6CF2EE2E6DE2EEE2402
:10608000FF2400E010E00E948B44823008F08AC0B8
:10609000F82DF03709F42BC5782D733709F4E1C4D6
:1060A00020E030E0C9012C960FB6F894DEBF0FBE99
:1060B000CDBFCF91DF911F910F91FF90EF90DF90B7
:1060C000CF90BF90AF909F908F907F906F905F9098
:1060D0004F903F902F900895282D233309F4FBC251
:1060E000282D372D462D552D642D732D822D992D5C
:1060F00003E3A02E11E7B12ECC24DD24EE24FF24EF
:1061000000E010E00E948B44823008F40DC2A82DFC
:10611000A43309F469C5E82DE03311F6F72DF23701
:1061200009F0BECF662009F0BBCF552009F0B8CFEB
:10613000442009F0B5CF332009F0B2CF222009F076
:10614000AFCF992009F0ACCF1092D3011092D201B9
:106150008091AD039091AE030E94DF1F82309105C4
:106160000CF4FDC58AEC92E00E94324C0E944E492C
:106170008B018091AD039091AE030E94DF1F8230AE
:10618000910554F08AEC92E00E94324C0E944E49F4
:106190000617170709F40DC68091A401882309F496
:1061A00057CF89C3B82DB93609F492C5382D323787
:1061B00009F076CF672D673609F072CF762D7037EC
:1061C00009F06ECF852D853709F06ACF442009F09C
:1061D00067CF332009F064CF222009F061CF9920E6
:1061E00009F05ECF00D086E292E0ADB7BEB712965E
:1061F0009C938E9311970E940B4E0F900F9080915D
:10620000A4010E94094388E10FB6F89480936000CE
:10621000109260000FBE83ED9CE1FC01E115F105D9
:1062200011F03197F1F78115910511F00197F1F710
:106230000C94007C21E030E035CFA82DA83709F080
:106240002FCFB72DB43709F02BCFE62DE13609F06B
:1062500027CF552009F024CF442009F021CF332047
:1062600009F01ECF222009F01BCF992009F018CF8A
:106270008091C40180FFABC381FFA9C38091470116
:10628000882309F490C586E391E000D000D023E98B
:1062900032E0ADB7BEB712963C932E931197149689
:1062A0009C938E9313970E940B4E809146010F9002
:1062B0000F900F900F90882309F472C586E391E048
:1062C00000D000D023E832E0EDB7FEB7328321835F
:1062D000948383830E940B4E0F900F900F900F902A
:1062E000019B5BC586E391E000D000D02FE632E051
:1062F000ADB7BEB712963C932E93119714969C930C
:106300008E9313970E940B4E0F900F900F900F904B
:1063100002994CC522E431E000D000D08BE592E038
:10632000EDB7FEB792838183348323830E940B4EA3
:106330000F900F900F900F9021E030E0B3CE882D9A
:10634000853609F0ADCE972D943609F0A9CE66209A
:1063500009F0A6CE552009F0A3CE442009F0A0CE26
:10636000332009F09DCE222009F09ACE992009F021
:1063700097CE8091A501882309F429C300D000D0CD
:106380008DE195E0EDB7FEB79283818381E090E0E7
:10639000948383830E940B4E8EE095E0ADB7BEB729
:1063A00012969C938E93119782E090E014969C93A2
:1063B0008E9313970E940B4E81E095E0EDB7FEB7E8
:1063C0009283818384E090E0948383830E940B4EC8
:1063D00084EF94E0ADB7BEB712969C938E9311975D
:1063E00088E090E014969C938E9313970E940B4E36
:1063F00082EE94E0EDB7FEB79283818380E190E076
:10640000948383830E940B4E8BEC94E0ADB7BEB7B0
:1064100012969C938E93119780E290E014969C9331
:106420008E9313970E940B4E80EC94E0EDB7FEB76D
:106430009283818380E490E0948383830E940B4E57
:1064400084EB94E0ADB7BEB712969C938E931197F0
:1064500080E890E014969C938E9313970E940B4EC5
:1064600086EA94E0EDB7FEB79283818380E091E005
:10647000948383830E940B4E8091D2019091D3012B
:106480002CE834E0ADB7BEB712963C932E9311972B
:1064900014969C938E9313970E940B4E0F900F901F
:1064A0000F900F908091AD039091AE030E94DF1F7B
:1064B0008230910564F08AEC92E060E070E040E1A7
:1064C00050E00E94244B7093D3016093D20100D01E
:1064D00081E791E1EDB7FEB7928381830E940B4E75
:1064E0008091D2019091D3010F900F9080FD72C4E2
:1064F0008091D2019091D30190FD60C48091D2012E
:106500009091D30183FFA4CD00D088EA93E0ADB78A
:10651000BEB712969C938E9311970E940B4E0F90CC
:106520000F9021E030E0BECD682D613309F441C306
:10653000882D823309F0B4CD972D913709F0B0CD75
:10654000662009F0ADCD552009F0AACD442009F010
:10655000A7CD332009F0A4CD222009F0A1CD9920A8
:1065600009F09ECD1092D3011092D20180901003B9
:1065700090901103A0901203B09013032091610139
:106580003091620140916301509164016091FC027D
:106590007091FD028091FE029091FF0269877A87D7
:1065A0008B879C8740900C0350900D0360900E03E6
:1065B00070900F03E0904801F090490100914A016A
:1065C00010914B013090DC0180912E0290912F02AE
:1065D000A0913002B091310289839A83AB83BC834E
:1065E0006091900270919102809192029091930239
:1065F0006D837E838F8398878DB79EB78C970FB6F8
:10660000F8949EBF0FBE8DBFEDB7FEB7319666EA18
:1066100071E0ADB7BEB712967C936E9311978282EC
:106620009382A482B5822683378340875187698508
:106630007A858B859C856287738784879587468654
:106640005786608A718AE28AF38A048B158B80915F
:10665000790190917A01A0917B01B0917C01868BA8
:10666000978BA08FB18F80917D0190917E01A09139
:106670007F01B0918001828F938FA48FB58F80911D
:10668000DD01868F178E30A211A28091DA019091E0
:10669000DB0193A382A389819A81AB81BC8184A30E
:1066A00095A3A6A3B7A36D817E818F81988560A7EE
:1066B00071A782A793A70E940B4E8091A401ADB74A
:1066C000BEB79C960FB6F894BEBF0FBEADBF882371
:1066D00009F4BECCF0C0372D313709F001CD66206A
:1066E00009F0FECC552009F0FBCC442009F0F8CC91
:1066F000332009F0F5CC222009F0F2CC992009F0E2
:10670000EFCC1092D3011092D2012091100330915E
:1067100011034091120350911303809190029091C4
:106720009102A0919202B0919302EDB7FEB73A9711
:106730000FB6F894FEBF0FBEEDBFEDB6FEB60894DF
:10674000E11CF11C67E971E072836183F701228328
:1067500033834483558386839783A087B1870E94C0
:106760000B4E8091A4012DB73EB7265F3F4F0FB669
:10677000F8943EBF0FBE2DBF882309F469CC9BC09F
:10678000772D7C3609F00CCC662009F009CC552019
:1067900009F006CC442009F003CC332009F000CCEA
:1067A000222009F0FDCB992009F0FACB8091C40199
:1067B00082FF0DC19091C30181E0911180E080932F
:1067C000C3018091C301882309F4DAC226E331E0D2
:1067D00000D000D08EEE91E0ADB7BEB712969C937C
:1067E0008E93119714963C932E9313970E940B4E01
:1067F0008091C3010F900F900F900F90882309F4A0
:10680000BBC25F9A21E030E04DCC872D823709F082
:10681000F4CA962D953609F0F0CA552009F0EDCA54
:10682000442009F0EACA332009F0E7CA222009F01F
:10683000E4CA992009F418CBE0CAA72DAF3609F0B5
:106840000ECCB62DBF3609F00ACCE52DE23609F0A4
:1068500006CC442009F003CC332009F000CC2220E0
:1068600009F0FDCB992009F0FACB0C94000021E04F
:1068700030E018CC372D313709F077CB662009F09E
:1068800074CB552009F071CB442009F06ECB332036
:1068900009F06BCB222009F068CB992009F065CB79
:1068A0001092D3011092D2010E9483228091A40100
:1068B000882309F4CDCB0E94094321E030E0F2CBDC
:1068C000372D313309F07DCA662D613709F079CA59
:1068D000552009F076CA442009F073CA332009F024
:1068E00070CA222009F06DCA992009F06ACAF8948A
:1068F00049E021E030E0F90140935700C895E02CD1
:1069000020E030E0F90140935700C895902C78942E
:10691000F89423E030E0F90140935700C895802CAB
:1069200082E090E0FC0140935700C895702C789469
:1069300000D000D000D041E253E0ADB7BEB7129610
:106940005C934E9311978091840290918502A0915F
:106950008602B0918702EDB7FEB783839483A58347
:10696000B6830E940B4E00D000D0EDB7FEB7319633
:106970004AEF52E0ADB7BEB712965C934E931197B3
:10698000728213828482158296821782E086118633
:106990000E940B4EEDB7FEB73A960FB6F894FEBFC5
:1069A0000FBEEDBFEAEBF3E020E4EF3FF20709F0A2
:1069B00098F480E090E005C030E4EF3FF30709F081
:1069C00068F431962081253CB9F70196F5CF0E94F5
:1069D000CA2821E030E066CB80E090E000D000D013
:1069E00028EE32E0ADB7BEB712963C932E931197C6
:1069F00014969C938E9313970E940B4E20916600E1
:106A0000EDB7FEB731968CED92E0ADB7BEB71296FA
:106A10009C938E931197228313820E940B4E809138
:106A2000C4009091C50021ED32E0EDB7FEB732838E
:106A30002183948383830E940B4E0F900F9081E7F4
:106A400091E1ADB7BEB712969C938E9311970E94B9
:106A50000B4E8091A4010F900F90882309F4F8CA7F
:106A60002ACF872D883709F01BCB962D943709F054
:106A700017CBA52DA13609F013CB442009F010CB7C
:106A8000332009F00DCB222009F00ACB992009F020
:106A900007CB8091C40181FF9ACF9091470181E09B
:106AA000911180E08093470180914701882309F488
:106AB00060C126E331E000D000D08AE292E0EDB779
:106AC000FEB792838183348323830E940B4E80918F
:106AD00047010F900F900F900F90882309F442C147
:106AE00081E090E00E94690A21E030E0DBCA272DB6
:106AF000283709F0D5CA362D343709F0D1CA652DAB
:106B0000613609F0CDCA442009F0CACA332009F021
:106B1000C7CA222009F0C4CA992009F0C1CA8091CD
:106B2000C40180FF54CF9091460181E0911180E033
:106B30008093460180914601882309F42BC126E306
:106B400031E000D000D084E492E0ADB7BEB7129639
:106B50009C938E93119714963C932E9313970E94B7
:106B60000B4E809146010F900F900F900F9088234D
:106B700009F409C181E090E00E94580A21E030E068
:106B800091CA272D233609F08BCA362D3D3609F0E0
:106B900087CA552009F084CA442009F081CA3320ED
:106BA00009F07ECA222009F07BCA992009F078CA30
:106BB0009ECE772D713709F073CA662009F070CA2E
:106BC000552009F06DCA442009F06ACA332009F043
:106BD00067CA222009F064CA992009F061CA10929C
:106BE000D3011092D2012DCAB72DB13709F058CA7E
:106BF000662009F055CA552009F052CA442009F010
:106C00004FCA332009F04CCA222009F049CA992002
:106C100009F046CA1092D3011092D201F6C9B72DDD
:106C2000BD3609F03DCA662009F03ACA552009F080
:106C300037CA442009F034CA332009F031CA22206F
:106C400009F02ECA992009F02BCA8091A50188234A
:106C500009F4BDCE2091600100D000D0EDB7FEB7A1
:106C600031968FEF91E0ADB7BEB712969C938E939D
:106C70001197228313820E940B4E0F900F900F905A
:106C80000F908091AD039091AE030E94DF1F823080
:106C9000910584F08AEC92E00E94324C0E945349A4
:106CA0006093600180E691E06CE170E041E050E0CB
:106CB0000E94D04E00D081E791E1EDB7FEB79283FC
:106CC00081830E940B4E0F900F9021E030E0EAC9C3
:106CD000E72DE33609F0E4C9F62DF33709F0E0C9F2
:106CE000252D2F3609F0DCC9442009F0D9C93320FD
:106CF00009F0D6C9222009F0D3C9992009F0D0C9DA
:106D00008091A501882309F462CE2091660000D00D
:106D100000D0EDB7FEB7319683EA92E0ADB7BEB7CB
:106D200012969C938E931197228313820E940B4E8E
:106D30000F900F900F900F908091AD039091AE0344
:106D40000E94DF1F823091050CF4B4CF8AEC92E0F0
:106D50000E94324C0E94534960936600ABCF0FEF04
:106D60001FEF07CA80E090E00E94690A21E030E04E
:106D700099C929E331E09FCE5F9821E030E092C9C4
:106D800029E331E025CD80E090E00E94580A21E01F
:106D900030E088C929E331E0D4CE89E391E0A4CA88
:106DA00089E391E08DCA89E391E06FCA2DE331E078
:106DB000B3CA1093DB010093DA01EEC900D084EF6F
:106DC00093E0EDB7FEB7928381830E940B4E0F9044
:106DD0000F9094CB00D08BE394E0ADB7BEB7129682
:106DE0009C938E9311970E940B4E0F900F9080CB27
:106DF0000F931F93CF93DF9300D000D000D087E58F
:106E000091E0EDB7FEB7928381838091CD0190919F
:106E1000CE01A091CF01B091D00183839483A5834B
:106E2000B6830E940B4E0F900F900F900F9001E7CA
:106E300011E1EDB7FEB7128301830E940B4E8DB7AF
:106E40009EB740970FB6F8949EBF0FBE8DBFCDB7CB
:106E5000DEB721968FE291E0EDB7FEB79283818392
:106E60006091220270912302809124029091250268
:106E700020E030E041E655E40E94E6486A837B83E7
:106E80008C839D838091880290918902A0918A02CF
:106E9000B0918B028E839F83A887B9878091C502AA
:106EA0009091C602A091C702B091C8028A879B87C1
:106EB000AC87BD8760911302709114028091150216
:106EC0009091160220E030E041E655E40E94E64849
:106ED0006E877F87888B998B0E940B4E8DB79EB7EC
:106EE00040960FB6F8949EBF0FBE8DBFEDB7FEB7AC
:106EF000128301830E940B4E8DB79EB740970FB649
:106F0000F8949EBF0FBE8DBFCDB7DEB7219687E048
:106F100091E0EDB7FEB79283818360912A02709170
:106F20002B0280912C0290912D0220E030E041E66E
:106F300055E40E94E6486A837B838C839D8380911D
:106F4000000390910103A0910203B09103038E838B
:106F50009F83A887B9878091320290913302A091D4
:106F60003402B09135028A879B87AC87BD876091D8
:106F7000040370910503809106039091070320E0BC
:106F800030E041E655E40E94E6486E877F87888BB3
:106F9000998B0E940B4E8DB79EB740960FB6F89412
:106FA0009EBF0FBE8DBFEDB7FEB7128301830E9457
:106FB0000B4E0F900F90DF91CF911F910F9108957D
:106FC000F89491E2E0E0F0E0909357008491E2E0E1
:106FD000F0E0909357002491E4E0F0E090935700A4
:106FE000E49190E0A0E0B0E0DC019927882730E050
:106FF00040E050E0542F432F322F2227820F931F5F
:10700000A41FB51F8E0F911DA11DB11D8093840279
:1070100090938502A0938602B09387027894089596
:107020002F923F924F925F926F927F928F929F9298
:10703000AF92BF92CF92DF92EF92FF920F931F9386
:10704000DF93CF93CDB7DEB72E970FB6F894DEBFA0
:107050000FBECDBF80E88093610082E08093610025
:107060000E94E0378091840290918502A09186026F
:10707000B0918702853027E992072EE1A20720E030
:10708000B20709F4F8C684E690E09093E00180939B
:10709000DF010E949B1281E00E94E7110E94914350
:1070A0008AE493E469E773E40E94524D02C00E94AF
:1070B00065430E945F438823D1F70E9495130E9485
:1070C00040228091D901882341F5209148013091D7
:1070D000490140914A0150914B0160E070E080EA23
:1070E00091E40E947D4826EA3BE944EC5CE30E947F
:1070F000354A2091690130916A0140916B015091AC
:107100006C010E947E489B01AC0120936101309389
:107110006201409363015093640180911D0381FDDE
:1071200093C680E090E07C0108C00894E11CF11C4B
:10713000B5E6EB16F10409F4A4C60E94A11F8091E4
:107140001D0381FFF2CF21E731E1ACEDB0E0BC835C
:10715000AB83E5ECF0E0FE83ED838AEA90E098876C
:107160008F83ABE9B0E0BA87A987ECE8F0E0FC8751
:10717000EB873E872D8702C00E94A11F80911D03CF
:1071800081FFFACF80911D038D7F80931D030E94A4
:107190003A1B0E945F43882379F38091AD0390915D
:1071A000AE030E94DF1F8130910509F4F3C08230E5
:1071B000910509F479C08330910509F4D5C0843074
:1071C000910509F4F0C08530910509F451C2AAE097
:1071D0002A2E332444245524662477248824992491
:1071E00000D0ED85FE85ADB7BEB71296FC93EE9349
:1071F00011970E940B4E0F900F909101A201B301C5
:10720000C4010E94A12E009709F0B6CF8091D80149
:10721000813009F422C3F22DF33709F45EC19101E4
:10722000A201B301C401F3E7AF2EE3E6BE2ECC24E6
:10723000DD24EE24FF2400E010E00E948B44823025
:10724000E0F5322D353709F456C39101A201B3019F
:10725000C40105E7A02EBB24CC24DD24EE24FF24AA
:1072600000E010E00E948B44823008F0C6C1822DFD
:10727000823609F43FC49101A201B301C40112E6B0
:10728000A12EBB24CC24DD24EE24FF2400E010E05A
:107290000E948B44823008F09FC3922D913609F4EE
:1072A0009EC50E94CA2868CF2090CA023324442475
:1072B000552466247724430193CFF22DF43709F443
:1072C000D3C29101A201B301C401F4E7AF2EEDE6F0
:1072D000BE2ECC24DD24EE24FF2400E010E00E942A
:1072E0008B44823008F012C1322D3C3609F4DCC3E5
:1072F0009101A201B301C4010CE6A02E14E6B12E47
:10730000CC24DD24EE24FF2400E010E00E948B4416
:10731000823008F086C3922D993619F6A32DA43633
:1073200009F0BFCF442009F0BCCF552009F0B9CFF8
:10733000662009F0B6CF772009F0B3CF882009F096
:10734000B0CF992009F0ADCF8091A501882309F431
:10735000A8CF31E03093DE018091A401882309F4A5
:107360000BCF0E94094308CFF091CA02FA83198219
:107370008091CB0229813A81280F311DC901190161
:10738000892F880F880B482E582E682E782E882E2D
:10739000982E26CF6091AF037091B0038AE090E001
:1073A0000E94DF4DE9CE2091CA0230E040E050E07B
:1073B00060E070E080E090E000E10E941A44122F4B
:1073C000F32EE42ED52EC62EB72EA82E292E2091D0
:1073D000CB0230E040E050E060E070E080E090E020
:1073E00008E00E941A44210FF1E0211708F0F0E0B4
:1073F0003F0DE1E03F1508F0E0E0F30FA1E0F317E7
:1074000008F0A0E0EA2B4E0D31E04E1508F030E018
:10741000E40FA1E0E41708F0A0E03A2B5D0DA1E035
:107420005D1508F0A0E0350F41E0351708F040E0A9
:10743000A42B6C0D51E06C1508F050E0A60F41E054
:10744000A61708F040E0542B7B0D41E07B1508F0B7
:1074500040E0570F61E0571708F060E0462B8A0DB7
:1074600061E08A1508F060E0480F71E0481708F005
:1074700070E0672B920D960F8091CC02820F61E035
:10748000821708F060E06F0F71E06F1708F070E08E
:107490007E0F21E07E1708F020E0E22FE30F21E0CD
:1074A000E31708F020E0322F3A0FF1E03A1708F026
:1074B000F0E0F50F21E0F51708F020E0240F51E08F
:1074C000241708F050E0282E362E472E5E2E632E0D
:1074D0007F2E822E952E990E83CE232D233609F0F2
:1074E0009ECE442009F09BCE552009F098CE662010
:1074F00009F095CE772009F092CE882009F08FCE42
:10750000992009F08CCE0E94F83626CF322D3536E0
:1075100009F40EC39101A201B301C401B5E6AB2E7B
:10752000A4E7BA2EF1E6CF2EE4E6DE2EEE24FF2409
:1075300000E010E00E948B44823008F001C2B22DBE
:10754000B33709F4A5C3F22DF33709F0AACE232DE2
:10755000243709F0A6CE442009F0A3CE552009F027
:10756000A0CE662009F09DCE772009F09ACE882023
:1075700009F097CE992009F094CE8091AD039091B7
:10758000AE030E94DF1F803191050CF44CC4F894C7
:107590008AEC92E00E94364C9093AC038093AB034C
:1075A0008FEC92E00E94364C8093AA0382ED92E029
:1075B0000E94364C8093A90385ED92E00E94364CE0
:1075C0008093A80388ED92E00E94364C8093A70335
:1075D0008BED92E00E94364C8093A603789400D005
:1075E000ED85FE85ADB7BEB71296FC93EE9311976D
:1075F0000E940B4E0F900F90AFCEE22DE33609F4B0
:10760000B0C29101A201B301C401B3E6AB2EA3E65F
:10761000BA2ECC24DD24EE24FF2400E010E00E94EA
:107620008B44823008F0ADC1222D263709F449C3BE
:10763000322D3D3609F035CE832D823609F031CE1C
:10764000442009F02ECE552009F02BCE662009F0FB
:1076500028CE772009F025CE882009F022CE992067
:1076600009F01FCEA1E0A093D8010E948D2884CDFF
:107670002091CA0230E040E050E060E070E080E03D
:1076800090E008E10E941A44122FF32EE42ED52E2A
:10769000C62EB72EA82E292E2091CB0230E040E036
:1076A00050E060E070E080E090E000E10E941A4469
:1076B000210FF1E0211708F0F0E03F0DE1E03F1568
:1076C00008F0E0E0F30FA1E0F31708F0A0E0EA2BE8
:1076D0004E0D31E04E1508F030E0E40FA1E0E41764
:1076E00008F0A0E03A2B5D0D41E05D1508F040E0A8
:1076F000350FA1E0351708F0A0E04A2B6C0D51E0E2
:107700006C1508F050E0460FA1E0461708F0A0E025
:107710005A2B7B0D61E07B1508F060E0570FA1E06C
:10772000571708F0A0E06A2B8A0D71E08A1508F05F
:1077300070E0680FA1E0681708F0A0E07A2B920DC6
:10774000970F1091CD02120F81E0121708F080E020
:10775000F82EFF0E81E0FF1608F080E0E82EEE0E16
:1077600081E0EE1608F080E0D82ED30E81E0D3162B
:1077700008F080E0C82EC40E81E0C41608F080E056
:10778000B82EB50E81E0B51608F080E0A82EA60E42
:1077900081E0A61608F080E0282E290E2091CC0268
:1077A00030E040E050E060E070E080E090E008E031
:1077B0000E941A44210FE1E0211708F0E0E0FF2DBC
:1077C000F30F31E0FF1508F030E0EF0FA1E0EF1705
:1077D00008F0A0E03A2B4E0DF1E04E1508F0F0E075
:1077E000340FA1E0341708F0A0E0FA2B5D0D41E062
:1077F0005D1508F040E0F50FA1E0F51708F0A0E0F6
:107800004A2B6C0D51E06C1508F050E0460FA1E0DA
:10781000461708F0A0E05A2B6B2D670F71E06B152F
:1078200008F070E0560FA1E0561708F0A0E07A2BA0
:107830008A0D61E08A1508F060E0780FA1E0781702
:1078400008F0A0E06A2B920D222E3E2E432E5F2ED2
:107850003A01872E962E990EC3CC9101A201B30155
:10786000C4010E94B22988CC232D2D3609F029CDE0
:10787000442009F026CD552009F023CD662009F0DB
:1078800020CD772009F01DCD882009F01ACD992050
:1078900009F017CD81E090918A01911180E08093E9
:1078A0008A01882309F4CDC231E03093D10186E307
:1078B00091E000D000D0ED81FE81ADB7BEB7129649
:1078C000FC93EE93119714969C938E9313970E94BA
:1078D0000B4E0F900F900F900F908AE891E062E4AA
:1078E00070E041E050E00E94D04E8091A4018823D6
:1078F00009F442CC36CD332009F0A7CC442009F05E
:10790000A4CC552009F0A1CC662009F09ECC7720AC
:1079100009F09BCC882009F098CC992009F095CCEF
:1079200060919402709195028091960290919702D5
:107930000E94C5098091A401882309F41DCC11CDB2
:10794000322D303709F48BC1B22DB43709F0A9CCF0
:10795000E32DE03709F0A5CCF42DF03709F0A1CCE8
:10796000252D2D3609F09DCC662009F09ACC772084
:1079700009F097CC882009F094CC992009F091CC9B
:1079800089CF922D993609F404C2B22DBC3609F084
:1079900088CCE32DE33609F084CC442009F081CC77
:1079A000552009F07ECC662009F07BCC772009F0C9
:1079B00078CC882009F075CC992009F072CC8091A0
:1079C000A501882309F46DCC1092DD018091A401FA
:1079D000882309F4D1CBC5CCA22DA83609F48EC1D9
:1079E000B22DB43709F05DCC332009F05ACC4420D5
:1079F00009F057CC552009F054CC662009F051CC41
:107A0000772009F04ECC882009F04BCC992009F062
:107A100048CC0E9432228091A401882309F4ACCB87
:107A2000A0CCB22DBD3609F481C1F22DF23609F099
:107A300038CC232D2D3609F034CC442009F031CC3C
:107A4000552009F02ECC662009F02BCC772009F0C8
:107A500028CC882009F025CC992009F022CC81E09F
:107A600090918B01911180E080938B01882309F420
:107A7000D4C186E391E000D000D0EF81F885ADB7A6
:107A8000BEB71296FC93EE93119714969C938E9327
:107A900013970E940B4E0F900F900F900F908BE852
:107AA00091E063E470E01DCF832D843609F020CC93
:107AB000442009F01DCC552009F01ACC662009F0AD
:107AC00017CC772009F014CC882009F011CC99202C
:107AD00009F00ECC8091A501882309F4E2CBF1E0F6
:107AE000F093DD010E9449128091A401882309F4DA
:107AF00043CB37CC332009F0BECB442009F0BBCBBD
:107B0000552009F0B8CB662009F0B5CB772009F0F5
:107B1000B2CB882009F0AFCB992009F0ACCB81E043
:107B200090E00E948F0988B191E0892788B924CB21
:107B3000832D843709F0EECC942D913609F0EACCF0
:107B4000A52DA43609F0E6CC662009F0E3CC772019
:107B500009F0E0CC882009F0DDCC992009F459CF58
:107B6000D9CCF32DF33609F04CCD442009F049CDA2
:107B7000552009F046CD662009F043CD772009F065
:107B800040CD882009F03DCD992009F03ACD00D0B4
:107B9000EB85FC85ADB7BEB71296FC93EE931197BB
:107BA0000E940B4EED85FE85ADB7BEB71296FC93D5
:107BB000EE9311970E940B4E80E090E0DC018093E1
:107BC000130290931402A0931502B09316028093AF
:107BD000C5029093C602A093C702B093C8028093D7
:107BE000880290938902A0938A02B0938B028093BB
:107BF000220290932302A0932402B0932502809343
:107C0000040390930503A0930603B09307038093A6
:107C1000320290933302A0933402B09335028093E2
:107C2000000390930103A0930203B0930303809396
:107C30002A0290932B02A0932C02B0932D028093E2
:107C4000CD019093CE01A093CF01B093D00180914C
:107C5000A4010F900F90882309F48ECA82CB832D44
:107C60008C3609F071CE942D953609F06DCEA52D88
:107C7000A83609F069CE662009F066CE772009F0B3
:107C800063CE882009F060CE992009F44CC05CCE08
:107C9000E32DE23709F057CC442009F054CC5520AD
:107CA00009F051CC662009F04ECC772009F04BCC7E
:107CB000882009F048CC992009F045CC0E94562034
:107CC0005BCA332009F0B4CC442009F0B1CC552074
:107CD00009F0AECC662009F0ABCC772009F0A8CC37
:107CE000882009F0A5CC992009F0A2CC0E9440225E
:107CF0008091A401882309F43FCA33CB332009F0D3
:107D00006FCE442009F06CCE552009F069CE662074
:107D100009F066CE772009F063CE882009F060CEA6
:107D2000992009F05DCE0E94DD2826CAE32DE536B4
:107D300009F07BCE442009F078CE552009F075CEAD
:107D4000662009F072CE772009F06FCE882009F006
:107D50006CCE992009F069CE81E09091A501911136
:107D600080E08093A501882309F45AC086E391E05E
:107D700000D000D02B813C81EDB7FEB73283218348
:107D8000948383830E940B4E0F900F900F900F905F
:107D9000F3C9A32DA33609F0F8CD442009F0F5CDA1
:107DA000552009F0F2CD662009F0EFCD772009F0DB
:107DB000ECCD882009F0E9CD992009F0E6CD80913D
:107DC000A501882309F46DCA1092DE0180918A0111
:107DD000882309F4C1CA21E02093D101BDCA332010
:107DE00009F05FCA442009F05CCA552009F059CA5D
:107DF000662009F056CA772009F053CA882009F096
:107E000050CA992009F04DCA80E090E00E948F0985
:107E100088B132E0832788B9AFC989E391E02BCEDE
:107E200089E391E0A5CF00D0E985FA85ADB7BEB76B
:107E30001296FC93EE9311970E940B4E0F900F90A9
:107E40008BCA89E391E035CD21E731E18CED90E0FB
:107E50009C838B83A5ECB0E0BE83AD83EAEAF0E0BF
:107E6000F887EF838BE990E09A878987ACE8B0E0E8
:107E7000BC87AB877EC98091C40188608093C401B0
:107E800002C980E090E00E948F0921E731E1ECED2A
:107E9000F0E0FC83EB8385EC90E09E838D83AAEA7F
:107EA000B0E0B887AF83EBE9F0E0FA87E9878CE8C8
:107EB00090E09C878B875DC989B1807408955E9A34
:107EC000569A08955E98569808955E98569A8DED44
:107ED00090E08115910511F00197F1F72FB7F89413
:107EE00056988EE190E08115910511F00197F1F718
:107EF00089B12FBF7894EEEBF0E0E115F10511F0B8
:107F00003197F1F74E9902C081E008958074089589
:107F10009FB7F894569AE0E0F0E0E115F10511F012
:107F20003197F1F781115698E5E0F0E0E115F105A0
:107F300011F03197F1F74E9B80E0E4E1F0E0E115BC
:107F4000F10511F03197F1F756989FBFEDE0F0E0A1
:107F5000E115F10511F03197F1F708950F931F9393
:107F6000182F08E0812F81700E94883F169581119B
:107F700010680150B9F7812F1F910F9108958FEF6D
:107F80000E94AE3F0895DF92EF92FF920F931F93EE
:107F9000CF93DF93182FEB010E94653F882359F0A0
:107FA000DD24DA948D2DDF91CF911F910F91FF90F9
:107FB000EF90DF90089580EF0E94AE3FDD2400E453
:107FC00098EFE92EE00E0BC0FF2061F580E00E94E3
:107FD000883F88818695888301500E15F9F081E0ED
:107FE0000E94883FF82E81E00E94883F882361F735
:107FF000FF2051F4011728F0888180FFE7CF101788
:1080000029F3D02EFF24F3948F2D0E94883F88817E
:1080100086958068888301500E1509F7002311F2B8
:108020002196CECF8EEFD82EBDCF0F931F93CF9337
:10803000DF93182FEB010E94653F209789F085E5BB
:108040000E94AE3F08E089910E94AE3F0150D9F7EF
:10805000812F0E94AE3FDF91CF911F910F91089524
:108060008CEC0E94AE3F812F0E94AE3FDF91CF91FA
:108070001F910F910895DC01CB0181159105A10598
:10808000B10529F081509040A040B040D9F7089543
:108090000F931F93CF93DF93FB01E801608170E0A2
:1080A000B181A0E06A2B7B2B803129F177FD34C0B0
:1080B000DA011C92883289F0CB01929582958F70FB
:1080C00089279F708927F90180836F70688380E01A
:1080D000DF91CF911F910F910895848190E0AC01C1
:1080E000407650704036510539F386FD1CC085FD41
:1080F0001CC0687FE1CFDB01AE7FAA0FBB1FAA0FB8
:10810000BB1FAA0FBB1F96816CE070E0691B710951
:108110006A0F7B1F77FFCCCF91E0DA019C937095BB
:1081200061957F4FC7CF6E7FC7CF6C7FC5CF0F9351
:108130001F93CF93DF938C01EB01FC018081BE0183
:108140000E94C33FF8018083982F91509D3F28F4EF
:108150009881983211F0903191F7DF91CF911F9172
:108160000F9108951F93CF93DF93EC010E94653F19
:1081700084EBBE010E94154081E00E94883F182FC9
:108180000E94653F81E0112309F480E0DF91CF91E7
:108190001F9108951F93CF93DF93182FEB010E9437
:1081A000653F0E945C3F882329F482E0DF91CF91F4
:1081B0001F91089584E4BE010E941540113039F0EA
:1081C0000E945F3F80E0DF91CF911F91089580E092
:1081D000DF91CF911F9108954F925F926F927F929E
:1081E0008F929F92AF92BF92CF92DF92EF92FF92C7
:1081F0000F931F93DF93CF93CDB7DEB729970FB6B9
:10820000F894DEBF0FBECDBF5C013B012A014901DE
:108210000E94653F8EEBB5010E9415408E010F5FF5
:108220001F4F78017AE0C72ED12CCC0EDD1E0E94A4
:10823000BF3FF70181937F01EC15FD05C1F7C80130
:1082400069E070E00E9465428823C1F083E02996CE
:108250000FB6F894DEBF0FBECDBFCF91DF911F9157
:108260000F91FF90EF90DF90CF90BF90AF909F90D5
:108270008F907F906F905F904F900895F50180816F
:10828000B801A301920184010E94484080E0DFCF41
:108290005F926F927F928F929F92AF92BF92CF9296
:1082A000DF92EF92FF920F931F93DF93CF93CDB79F
:1082B000DEB729970FB6F894DEBF0FBECDBF582E9C
:1082C0004B013A0159018EEB60E070E00E941540CD
:1082D0008E010F5F1F4F7801EAE0CE2ED12CCC0E1D
:1082E000DD1E0E94BF3FF70181937F01EC15FD0564
:1082F000C1F7C80169E070E00E9465428823B9F0C7
:1083000083E029960FB6F894DEBF0FBECDBFCF91A4
:10831000DF911F910F91FF90EF90DF90CF90BF9072
:10832000AF909F908F907F906F905F900895852D74
:10833000B801A401930185010E94484080E0E1CF8B
:10834000EF92FF920F931F93DF93CF93CDB7DEB7DA
:1083500028970FB6F894DEBF0FBECDBF182F062F9B
:108360007E010894E11CF11CC701A4EBB1E038E0E8
:108370000D90FC010192CF013150D1F7242F33270A
:1083800027FD309541E752E0249FC001259F900DC5
:10839000349F900D112464E670E00E94B84AAB014E
:1083A00064E6069FB0011124460F571FF701CE0166
:1083B0000996619170E026173707B1F0E817F907C1
:1083C000C1F7112319F0509541955F4FCA012896C6
:1083D0000FB6F894DEBF0FBECDBFCF91DF911F91D6
:1083E0000F91FF90EF9008954F5F5F4FEACF0F938B
:1083F0001F93DF93CF93CDB7DEB72B970FB6F894CB
:10840000DEBF0FBECDBF182F092F885F612F792FD8
:108410000E94CA40882371F064E371E2CB012B967D
:108420000FB6F894DEBF0FBECDBFCF91DF911F9185
:108430000F9108956AE673E883E090E00E943B4064
:10844000812F902FBE016F5F7F4FAE014E5F5F4F58
:108450009E012D5F3F4F0E94EC408823E9F69E016C
:108460002C5F3F4FD901ECEAF1E088E001900D92DA
:108470008150E1F74B81E42FF0E061E772E0E69F85
:10848000C001E79F900DF69F900D112464E670E007
:108490000E94B84A9A8184E6989FC0011124680F0F
:1084A000791FF901CE010C962191421759F0E81776
:1084B000F907D1F78981882309F4B0CF70956195C8
:1084C0007F4FACCF6F5F7F4FF5CF61157105E1F046
:1084D000E82FF92F20E030E080E0A8E1419198E01A
:1084E00004C08695915051F04695542F582750FF5F
:1084F000F8CF8A27869580689150B1F72F5F3F4F5C
:108500006217730759F7089580E008951F920F923C
:108510000FB60F920BB60F9211248F93EF93FF9328
:108520008091C600E0912203F0E0EF73F070ED5D02
:10853000FC4F8083809122038F5F80932203FF9101
:10854000EF918F910F900BBE0F900FBE0F901F9069
:1085500018951F920F920FB60F920BB60F9211241F
:108560008F939F93EF93FF939091630380916503A3
:108570009817D1F0E0916503F0E0EF73F070EA59DD
:10858000FC4F80818093C600809165038F5F80934C
:108590006503FF91EF919F918F910F900BBE0F900C
:1085A0000FBE0F901F9018958091C1008F7D809312
:1085B000C100EFCF161617061CF5DC0120E030E0F5
:1085C00090912203809164039817D1F3E0916403A2
:1085D000F0E0EF73F070ED5DFC4F4081809164033B
:1085E0008F5F809364034D93CD014D3029F02F5F51
:1085F0003F4F2617370724F3FC011082C901089565
:1086000020E030E0F9CF8091630390916503891BEE
:10861000089540E450E09091630320916503921B1C
:108620009A01291B310923303105ACF3E091630332
:10863000F0E0EF73F070EA59FC4F808380916303A0
:108640008F5F809363038091C10080628093C1003B
:108650000895CF93DF93EC01FC018491882341F0CE
:1086600021960E940943FE01219684918823C9F72F
:10867000DF91CF910895CF93DF93EC018881882318
:1086800031F021960E94094389918823D9F7DF911F
:10869000CF9108951F93182F8A3039F0812F0E94AF
:1086A000094380E090E01F9108958DE00E94094306
:1086B000812F0E94094380E090E01F9108958091EE
:1086C000220390916403891B089590912203809165
:1086D00064039817D1F3E0916403F0E0EF73F07056
:1086E000ED5DFC4F8081909164039F5F90936403E4
:1086F000089590912203809164039817D1F3E0913B
:108700006403F0E0EF73F070ED5DFC4F80819091B9
:1087100064039F5F9093640390E008950E9409436F
:10872000089585E090E09093C5008093C40082E0B6
:108730008093C0008AE98093C10008958091A603C8
:108740008F5F8093A6038C3309F008951092A603DF
:108750008091A7038F5F8093A7038C33B1F71092AA
:10876000A7038091A8038F5F8093A803883169F7DE
:108770001092A8038091A9038F5F8093A903803290
:10878000B9F08F31F1F08E3169F18D31B1F1809115
:10879000AA038D30D1F681E08093AA038091AB03C8
:1087A0009091AC0301969093AC038093AB03089532
:1087B0008091AA038F5F8093AA0391E09093A9030D
:1087C000E8CF8091AA03843031F0863021F08930DF
:1087D00011F08B30F1F68F5F8093AA0391E09093B4
:1087E000A903D7CF8091AA03823099F683E08093C2
:1087F000AA0381E08093A90308958091AA0382309F
:1088000041F64091AB03E091AC03842F9E2F64E6C8
:1088100070E00E94A44A009751F4842F9E2F60E9D3
:1088200071E00E94A44A882309F48FCFDFCF842F00
:108830008370F9CF0F93DF93CF93CDB7DEB76097F7
:108840000FB6F894DEBF0FBECDBF002309F459C0A8
:1088500029833A834B835C836D837E838F839887E0
:10886000E0E2E01B29813A814B815C811E16BCF05D
:1088700019861A861B861C868E2F992787FD909550
:10888000909581959F4F04C0220F331F441F551FA1
:108890008A95D2F72D873E874F87588B2AC0CA0109
:1088A000B901002E04C0660F771F881F991F0A9414
:1088B000D2F769877A878B879C87DA01C90104C060
:1088C000B695A79597958795EA95D2F72D813E8124
:1088D0004F81588504C0220F331F441F551F0A952E
:1088E000D2F7822B932BA42BB52B8D879E87AF8736
:1088F000B88B29853A854B855C856D857E858F850E
:10890000988960960FB6F894DEBF0FBECDBFCF91A9
:10891000DF910F910895A0E1B0E0E1E9F4E40C9457
:10892000F54A29833A834B835C836D837E838F83EF
:108930009887A986BA86CB86DC86ED86FE860F8769
:10894000188B2D813E814F8158858D859E85AF8501
:10895000B889281739074A075B07C8F082179307B9
:10896000A407B50790F029813A814B815C81898504
:108970009A85AB85BC85281739074A075B0738F00D
:1089800082179307A407B50720F482E003C080E0B4
:1089900001C081E06096EAE00C94114B2F923F9267
:1089A0004F925F926F927F928F929F92AF92BF92FF
:1089B000CF92DF92EF92FF920F931F93DF93CF93AB
:1089C000CDB7DEB763970FB6F894DEBF0FBECDBF4D
:1089D0006C017F876E87FC0117821682838181FD7F
:1089E00004C06FC34C855D8504C01E010894211C22
:1089F000311CF6019381EE85FF8593FD859193FFF0
:108A00008191FF87EE87882309F457C3853241F4AB
:108A100093FD859193FF8191FF87EE87853259F40D
:108A200090E0B6014A8B5B8B0E94DF4D4A895B89DF
:108A30005D874C87D7CF10E0FF2400E00032B0F410
:108A40008B3269F08C3228F4803251F0833271F429
:108A50000BC08D3239F0803349F401602CC00260C4
:108A6000046029C0086027C0006125C007FD2EC032
:108A7000282F20532A3098F406FF08C0812F880F32
:108A8000182F110F110F180F120F15C08F2D880FEF
:108A9000F82EFF0CFF0CF80EF20E00620CC08E32A6
:108AA00021F406FD0AC3006406C08C3611F4006888
:108AB00002C0883659F4EE85FF8593FD859193FFBA
:108AC0008191FF87EE87882309F0B8CF982F9554BE
:108AD000933018F40061805E06C0982F955693304D
:108AE00008F09BC10F7E06FF16E06FE3E62EE02242
:108AF000853619F4F0E4EF2A07C0863619F420E829
:108B0000E22A02C011111150E7FE06C01C3340F4E6
:108B1000912E939427E00BC0183030F4212F06C01B
:108B200027E03CE3932E03C027E017E09924CA0115
:108B300004969D878C87FA0160817181828193817F
:108B4000A101092D0E94544C5C016980262D30E062
:108B5000398B288B60FE03C0388933FF06C0E1FCE7
:108B600006C0E2FE06C000E205C00DE203C00BE253
:108B700001C000E0888999898C7090700097C1F1DC
:108B8000002311F084E001C083E08F1558F4F81A37
:108B9000E3FC09C080E290E0B6010E94DF4DFA9448
:108BA000C9F701C0FF24002329F0802F90E0B6010F
:108BB0000E94DF4D888983FD03C007E711E10EC0E5
:108BC00003E711E10BC0A114B10409F0805290E059
:108BD000B6010E94DF4D0F5F1F4F05C0AE2CBB24B6
:108BE00090E1A922BB24F8018491882361F762C235
:108BF000E7FE0EC09A0CF889F4FF04C08A81813325
:108C000009F49A94191454F5292D293050F52DC0E2
:108C1000E6FC2BC0812F90E08A159B054CF03CEFC1
:108C2000A3163FEFB30624F080E8E82A01C01150F4
:108C3000112349F0E2E0F0E0EC0FFD1FE10FF11D20
:108C400080818033A1F3E7FE10C0912E9394812F91
:108C500090E0A816B90644F41A1907C09924939411
:108C600004C098E0992E01C010E0E7FE07C01A1476
:108C70001B043CF495012F5F3F4F05C025E030E019
:108C800002C021E030E0002311F02F5F3F4F11239D
:108C900029F0812F90E00196280F391F8F2D90E049
:108CA0002817390714F4F21A01C0FF244E2C55245A
:108CB000C20189709070009749F406C080E290E08C
:108CC000B6010E94DF4DFA94FF20C1F7002329F07E
:108CD000802F90E0B6010E94DF4D43FC09C006C022
:108CE00080E390E0B6010E94DF4DFA94FF20C1F7C7
:108CF000E7FE46C03501B7FE02C066247724250191
:108D00000894411C511C46185708420C531CF5018D
:108D1000E919F1094F01812F90E000271127081B65
:108D2000190BFFEF6F16FFEF7F0629F48EE290E03C
:108D3000B6010E94DF4DA614B70434F086149704E0
:108D40001CF4F201808101C080E30894610871087D
:108D50000894411C511C601671062CF090E0B6017D
:108D60000E94DF4DDECF6A147B0441F49A81963372
:108D700020F4953319F4F889F4FF81E390E049C0B9
:108D80008A81813311F02FEE622290E0B6010E94B9
:108D9000DF4D112389F08EE290E0B6010E94DF4D95
:108DA00002E0F101E00FF11D0F5F808190E0B6015C
:108DB0000E94DF4D1150A9F744FE03C085E490E006
:108DC00002C085E690E0B6010E94DF4DB7FC05C009
:108DD000A114B10441F464FE06C0B094A194B1089A
:108DE000B3948DE201C08BE290E0B6010E94DF4DAA
:108DF00080E305C08F5FE6EFFFEFAE0EBF1EFAE027
:108E0000AF16B104BCF790E0B6010E94DF4DC5017A
:108E1000C096B6010E94DF4D4DC1833631F08337D5
:108E200089F0833509F059C022C09A012E5F3F4F67
:108E30003D872C87FA0180818983310181E0A82E4A
:108E4000B12C13C09A012E5F3F4F3D872C87FA014A
:108E50006080718006FF03C0612F70E002C06FEF79
:108E60007FEFC3010E943F4D5C010F7714C09A0150
:108E70002E5F3F4F3D872C87FA016080718006FF8F
:108E800003C0612F70E002C06FEF7FEFC3010E944B
:108E9000344D5C01006803FD1CC006C080E290E018
:108EA000B6010E94DF4DFA948F2D90E0A816B90606
:108EB000A8F30FC0F30107FD859107FF81913F01E2
:108EC00090E0B6010E94DF4DF110FA940894A108D9
:108ED000B108A114B10471F7EDC0843611F08936E0
:108EE00061F507FF0BC09A012C5F3F4F3D872C8730
:108EF000FA0160817181828193810CC09A012E5F99
:108F00003F4F3D872C87FA0160817181882777FD6B
:108F10008095982F0F7697FF08C090958095709553
:108F200061957F4F8F4F9F4F0068A1012AE030E08D
:108F30000E94624E982E921841C0853721F40F7E10
:108F40002AE030E020C0097F8F36A9F0803720F476
:108F5000883509F0B2C00BC0803721F0883709F09E
:108F6000ACC001C0006104FF09C0046007C004FF79
:108F700008C0066006C028E030E005C020E130E00F
:108F800002C020E132E007FF0AC0CA0104969D87B3
:108F90008C87FA01608171818281938109C0CA0145
:108FA00002969D878C87FA016081718180E090E054
:108FB000A1010E94624E982E92180F7706FF09C0F9
:108FC0000E7F911630F404FF06C002FD04C00F7E30
:108FD00002C0E92C01C0E12E802F90E004FF0CC0FC
:108FE000FE01E90DF11D2081203311F4097E09C035
:108FF000E39402FF06C004C086789070009709F0E1
:10900000E394A02EBB2403FD14C000FF0FC0EF1497
:1090100028F4192D1F0D1E19EF2C08C0192D06C09C
:1090200080E290E0B6010E94DF4DE394EF14C0F3BC
:1090300004C0EF1410F4FE1801C0FF24A4FE0FC0FA
:1090400080E390E0B6010E94DF4DA2FE1FC0A1FEAA
:1090500003C088E590E010C088E790E00DC0C5012E
:1090600086789070009791F0A1FC02C080E201C068
:109070008BE207FD8DE290E0B6010E94DF4D06C055
:1090800080E390E0B6010E94DF4D11509116C0F3CD
:109090009A94F101E90DF11D808190E0B6010E94E2
:1090A000DF4D9920A9F706C080E290E0B6010E944A
:1090B000DF4DFA94FF20C1F795CCF6012681378168
:1090C00002C02FEF3FEFC90163960FB6F894DEBFE1
:1090D0000FBECDBFCF91DF911F910F91FF90EF9009
:1090E000DF90CF90BF90AF909F908F907F906F90C8
:1090F0005F904F903F902F9008955058BB27AA271C
:109100000ED075C166D130F06BD120F031F49F3FA5
:1091100011F41EF45BC10EF4E095E7FB51C1E92F99
:1091200077D180F3BA17620773078407950718F0A1
:1091300071F49EF58FC10EF4E0950B2EBA2FA02D81
:109140000B01B90190010C01CA01A0011124FF27F4
:10915000591B99F0593F50F4503E68F11A16F040EF
:10916000A22F232F342F4427585FF3CF46953795EE
:109170002795A795F0405395C9F77EF41F16BA0BB3
:10918000620B730B840BBAF09150A1F0FF0FBB1F61
:10919000661F771F881FC2F70EC0BA0F621F731FAA
:1091A000841F48F4879577956795B795F7959E3F07
:1091B00008F0B3CF9395880F08F09927EE0F979595
:1091C00087950895D9D008F481E008950CD00FC197
:1091D00007D140F0FED030F021F45F3F19F0F0C02D
:1091E000511139C1F3C014D198F39923C9F3552310
:1091F000B1F3951B550BBB27AA276217730784078A
:1092000038F09F5F5F4F220F331F441FAA1FA9F33F
:1092100033D00E2E3AF0E0E830D091505040E69531
:10922000001CCAF729D0FE2F27D0660F771F881F92
:10923000BB1F261737074807AB07B0E809F0BB0B81
:10924000802DBF01FF2793585F4F2AF09E3F5105A5
:1092500068F0B6C000C15F3FECF3983EDCF3869542
:1092600077956795B795F7959F5FC9F7880F911D1B
:109270009695879597F90895E1E0660F771F881F07
:10928000BB1F621773078407BA0720F0621B730BBA
:10929000840BBA0BEE1F88F7E095089504D068940C
:1092A000B111D9C00895BCD088F09F5790F0B92F64
:1092B0009927B751A0F0D1F0660F771F881F991F2B
:1092C0001AF0BA95C9F712C0B13081F0C3D0B1E03D
:1092D0000895C0C0672F782F8827B85F39F0B93F4D
:1092E000CCF3869577956795B395D9F73EF490952D
:1092F0008095709561957F4F8F4F9F4F0895E894AB
:1093000009C097FB3EF490958095709561957F4FCD
:109310008F4F9F4F9923A9F0F92F96E9BB2793957B
:10932000F695879577956795B795F111F8CFFAF48B
:10933000BB0F11F460FF1BC06F5F7F4F8F4F9F4FBC
:1093400016C0882311F096E911C0772321F09EE81A
:10935000872F762F05C0662371F096E8862F70E080
:1093600060E02AF09A95660F771F881FDAF7880F5A
:109370009695879597F90895990F0008550FAA0BB0
:10938000E0E8FEEF16161706E807F907C0F0121618
:109390001306E407F50798F0621B730B840B950B1B
:1093A00039F40A2661F0232B242B252B21F4089570
:1093B0000A2609F4A140A6958FEF811D811D08950D
:1093C00097F99F6780E870E060E008959FEF80EC78
:1093D000089500240A94161617061806090608951B
:1093E00000240A9412161306140605060895092E81
:1093F0000394000C11F4882352F0BB0F40F4BF2BF0
:1094000011F460FF04C06F5F7F4F8F4F9F4F08952F
:1094100057FD9058440F551F59F05F3F71F0479525
:10942000880F97FB991F61F09F3F79F0879508950A
:10943000121613061406551FF2CF4695F1DF08C029
:10944000161617061806991FF1CF86957105610546
:1094500008940895E894BB2766277727CB0197F9EE
:1094600008958ADF08F48FEF08950BD0C0CFB1DFE5
:1094700028F0B6DF18F0952309F0A2CFA7CF11246A
:10948000EACFC6DFA0F3959FD1F3950F50E0551FAB
:10949000629FF001729FBB27F00DB11D639FAA2749
:1094A000F00DB11DAA1F649F6627B00DA11D661F98
:1094B000829F2227B00DA11D621F739FB00DA11DB9
:1094C000621F839FA00D611D221F749F3327A00D73
:1094D000611D231F849F600D211D822F762F6A2F0F
:1094E00011249F5750408AF0E1F088234AF0EE0F94
:1094F000FF1FBB1F661F771F881F91505040A9F7A1
:109500009E3F510570F05CCFA6CF5F3FECF3983ED5
:10951000DCF3869577956795B795F795E7959F5F07
:10952000C1F7FE2B880F911D9695879597F90895A1
:10953000991B79E004C0991F961708F0961B881FA5
:109540007A95C9F780950895AA1BBB1B51E107C006
:10955000AA1FBB1FA617B70710F0A61BB70B881FC3
:10956000991F5A95A9F780959095BC01CD01089552
:1095700097FB092E07260AD077FD04D0E5DF06D039
:1095800000201AF4709561957F4F0895F6F7909535
:1095900081959F4F0895A1E21A2EAA1BBB1BFD01C6
:1095A0000DC0AA1FBB1FEE1FFF1FA217B307E407C2
:1095B000F50720F0A21BB30BE40BF50B661F771F1A
:1095C000881F991F1A9469F76095709580959095FA
:1095D0009B01AC01BD01CF0108952F923F924F92A4
:1095E0005F926F927F928F929F92AF92BF92CF9233
:1095F000DF92EF92FF920F931F93CF93DF93CDB73C
:10960000DEB7CA1BDB0B0FB6F894DEBF0FBECDBFB3
:1096100009942A88398848885F846E847D848C8484
:109620009B84AA84B984C884DF80EE80FD800C818D
:109630001B81AA81B981CE0FD11D0FB6F894DEBF70
:109640000FBECDBFED0108952F923F924F925F92D2
:109650006F927F929F92AF92BF92CF92DF92EF92E2
:10966000FF920F931F93CF93DF933B01EA016115A4
:10967000710519F0FB0180839183209739F09E01D9
:10968000225030402332310508F0D5C0C82ED92EE3
:10969000F60111916F017F01812F90E00E942C4D06
:1096A0000097B1F71D3231F4F60111917F01992431
:1096B000939406C01B3219F4F60111917F0199248D
:1096C000209719F0C031D105D1F4103389F4F70196
:1096D0008081883711F0883559F4F701118182E0D3
:1096E00090E0E80EF91E92E0992AC0E1D0E007C0B0
:1096F000209729F41033B1F0CAE0D0E02BC0CA3073
:10970000D10541F1C031D10521F0C830D105A9F40E
:1097100009C02FEFA22E2FEFB22E2FEFC22E2FE077
:10972000D22E20C0C8E0D0E09FEFA92E9FEFB92E27
:109730009FEFC92E9FE1D92E15C09E01442737FD0A
:109740004095542F6FEF7FEFCB010E94CB4A590118
:109750006A0108C089E9A82E89E9B82E89E9C82ECE
:1097600089E1D82E60E020E030E0A9011E01442408
:1097700037FC4094542C012F00530A3060F0812FA5
:1097800081548A3110F4075006C0812F81568A31E6
:1097900050F5012F0755802F90E08C179D071CF581
:1097A0006F3FE9F0A216B306C406D506A8F0CA01B9
:1097B000B901A20191010E94F0519B01AC01802FDF
:1097C00090E0A0E0B0E0280F391F4A1F5B1F281768
:1097D00039074A075B0710F46FEF01C061E0F7013A
:1097E00011917F01C8CF6114710481F0662339F0B3
:1097F0000894E108F108F301F182E08207C091FECC
:1098000005C0C7010297F3019183808390FE07C0D2
:1098100050954095309521953F4F4F4F5F4F67FFD3
:109820000DC082E290E09093B4038093B3032FEFD6
:109830003FEFA90103C020E030E0A901B901CA014E
:10984000DF91CF911F910F91FF90EF90DF90CF901C
:10985000BF90AF909F907F906F905F904F903F90A0
:109860002F900895662777270C944050FC01882795
:109870009927E89421912032E9F3293010F02E3015
:10988000C8F32B3241F02D3239F4689404C00E94A1
:109890004A4D820F911D219120532A30C0F31EF4AE
:1098A000909581959F4F0895283008F027E0332741
:1098B000DA01990F311D87FD9160009661057105F0
:1098C00039F432602E5F3D9330E32A95E1F7089535
:1098D0009F3F30F080387105610509F03C5F3C5FC7
:1098E0003D93913008F08068911DDF93CF931F93D3
:1098F0000F93FF92EF92192F987F9695E92F9695E7
:109900009695E90FFF27EB52FE4E99273327EE2459
:10991000FF24A701E70105900894079428F4360F67
:10992000E71EF81E491F511D660F771F881F991FDC
:109930000694A1F70590079428F4E70EF81E491F36
:10994000561FC11D770F881F991F661F0694A1F728
:109950000590079428F4F80E491F561FC71FD11D04
:10996000880F991F661F771F0694A1F7059007942B
:1099700020F4490F561FC71FD81F990F661F771F66
:10998000881F0694A9F784911095177041F0D69519
:10999000C79557954795F794E7941A95C1F7EBE764
:1099A000F1E1689415901591359165919591059027
:1099B0007FE27395E118F10A430B560BC90BD009EE
:1099C000C0F7E10CF11E431F561FC91FD01D7EF4C6
:1099D000703311F48A95E6CFE894015030F0080F07
:1099E0000AF40027021708F4202F2395022F7A3358
:1099F00028F079E37D932A95E9F710C07D932A95A5
:109A000089F6069497956795379517951794E118F9
:109A1000F10A430B560BC90BD00998F023957E91A0
:109A200073957A3308F070E37C932013B8F77E9136
:109A300070617D9330F0839571E37D9370E32A9597
:109A4000E1F71124EF90FF900F911F91CF91DF91DB
:109A5000992787FD909508959111A0C4803219F03F
:109A600089508550D0F70895FC01059061507040F1
:109A70000110D8F7809590958E0F9F1F0895FC01D7
:109A80006150704001900110D8F7809590958E0F2D
:109A90009F1F08957AE0979F902D879F802D910DAD
:109AA000112408950F931F93CF93DF938C01EB0143
:109AB000009711F42097C9F181E090E06EE070E02A
:109AC0000E94E84EFC019C01009789F180E88383A5
:109AD000209771F0D387C28781E883838091AD039B
:109AE0009091AE03009721F4F093AE03E093AD03A1
:109AF00001151105E1F0118700878381826083835E
:109B00008091AF039091B003009789F4F093B00374
:109B1000E093AF038091B1039091B203009739F4C1
:109B2000F093B203E093B10302C020E030E0C9013A
:109B3000DF91CF911F910F910895CF93DF93EC01A7
:109B40003B8130FF36C036FF09C03F7B3B838E81AF
:109B50009F8101969F838E832A8129C032FF0FC087
:109B6000E881F9818081992787FD9095009719F404
:109B700030623B831EC03196F983E88311C0EA85C9
:109B8000FB85CE01099597FF0BC02B813FEF8F3FDF
:109B9000930711F480E101C080E2822B8B8309C01E
:109BA0002E813F812F5F3F4F3F832E83282F30E050
:109BB00002C02FEF3FEFC901DF91CF9108950F93BE
:109BC0001F93CF93DF938C01EB018B8181FF1BC02F
:109BD00082FF0DC02E813F818C819D81281739071E
:109BE00064F4E881F9810193F983E88306C0E8858C
:109BF000F985802F0995009731F48E819F81019618
:109C00009F838E8302C00FEF1FEFC801DF91CF91BA
:109C10001F910F910895DF93CF93CDB7DEB7FE016B
:109C20003596619171918091AF039091B003DC0101
:109C300013962C911397286013962C93AF010E94D2
:109C4000CE44E091AF03F091B0032381277F2383BB
:109C5000CF91DF910895EF92FF920F931F93CF93CF
:109C6000DF938C01E091AF03F091B003838181FF1A
:109C70001FC0C0E0D0E00AC0DB011896ED91FC9156
:109C800019970995009711F0CFEFDFEFF801819157
:109C90008F016091AF037091B003882369F7DB01F6
:109CA0001896ED91FC9119978AE00995009711F0AB
:109CB000CFEFDFEFCE01DF91CF911F910F91FF909A
:109CC000EF900895FA01AA27283051F1203181F14F
:109CD000E8946F936E7F6E5F7F4F8F4F9F4FAF4FB4
:109CE000B1E03ED0B4E03CD0670F781F891F9A1FC7
:109CF000A11D680F791F8A1F911DA11D6A0F711D7B
:109D0000811D911DA11D20D009F468943F912AE086
:109D1000269F11243019305D3193DEF6CF0108956E
:109D2000462F4770405D4193B3E00FD0C9F7F6CF9F
:109D3000462F4F70405D4A3318F0495D31FD405267
:109D4000419302D0A9F7EACFB4E0A69597958795FD
:109D500077956795BA95C9F70097610571050895DC
:109D60009B01AC010A2E0694579547953795279588
:109D7000BA95C9F7620F731F841F951FA01D089520
:109D8000DC01CB01FC01F999FECF06C0F2BDE1BDBB
:109D9000F89A319600B40D9241505040B8F70895AA
:109DA000DC01CB0103C02D910E94DB4E415050409D
:109DB000D0F70895262FF999FECF1FBA92BD81BD25
:109DC00020BD0FB6F894FA9AF99A0FBE019608953D
:109DD000EF92FF920F931F93CF93DF93689F8001C1
:109DE000699F100D789F100D1124C8010E940D4F1E
:109DF000E82EE7017E01F92EE701209731F08E2D44
:109E000060E070E0A8010E94E951CE01DF91CF919E
:109E10001F910F91FF90EF900895CF93DF938230C1
:109E2000910510F482E090E0E091B703F091B8035F
:109E300040E050E020E030E026C06081718168178A
:109E40007907E0F06817790781F482819381211501
:109E5000310531F0D90113969C938E9312972BC044
:109E60009093B8038093B70326C04115510519F0AC
:109E70006417750718F4AB01E901DF019F017281D6
:109E80006381E72FF62F3097C1F64115510501F197
:109E9000481B590B4430510580F412968D919C91CA
:109EA0001397209719F09B838A8304C09093B8037B
:109EB0008093B703FD01329646C0FD01E40FF51F04
:109EC000819391934250504011965C934E933BC0C6
:109ED0002091B5033091B6032115310541F420914D
:109EE000BE013091BF013093B6032093B50320919A
:109EF000C0013091C1012115310541F42DB73EB7A4
:109F00004091BC015091BD01241B350BE091B5037C
:109F1000F091B603E217F307A0F42E1B3F0B2817AE
:109F2000390778F0AC014E5F5F4F2417350748F0D2
:109F30004E0F5F1F5093B6034093B50381939193E7
:109F400002C0E0E0F0E0CF01DF91CF910895CF9320
:109F5000DF93009709F491C0FC01329713821282BB
:109F60006091B7037091B8036115710581F4208188
:109F70003181280F391F8091B5039091B603821764
:109F8000930799F5F093B603E093B50376C0DB0130
:109F900080E090E002C0CD01D901AE17BF0748F4C0
:109FA00012962D913C91139721153105A1F7CD0102
:109FB00021C0B383A283EF01499159919E01240FDF
:109FC000351FA217B30779F42D913C911197240FF7
:109FD000351F2E5F3F4F3183208312962D913C9188
:109FE000139733832283009729F4F093B803E09307
:109FF000B70343C0DC011396FC93EE9312974D9187
:10A000005D91A40FB51FEA17FB0769F42081318128
:10A01000240F351F2E5F3F4FEC01398328832281A7
:10A0200033813B832A83E0E0F0E002C0FB01BC0106
:10A03000DB0112968D919C9113970097B9F79B01C4
:10A040002E5F3F4F8D919C911197820F931F4091EE
:10A05000B5035091B6034817590779F4309729F49E
:10A060001092B8031092B70302C0138212822250DA
:10A0700030403093B6032093B503DF91CF9108951C
:10A080006F927F928F929F92AF92BF92CF92DF9208
:10A09000EF92FF920F931F93DF93CF930F92CDB761
:10A0A000DEB75B016115710521F0DB018C93119620
:10A0B0009C93482F592F6A01F601E1906F018F019F
:10A0C0008E2D90E00E942C4D0097B1F7FE2DFD32B1
:10A0D00029F4D601ED908D0121E007C0BE2DBB32E1
:10A0E00019F4F601E1908F0120E068010894C1089D
:10A0F000D108C60165E772E143E050E029830E9480
:10A10000D1512981009711F572E0E72EF12CE00E74
:10A11000F11EC70168E772E145E050E00E94D151AD
:10A120002981009729F467E0E62EF12CE00EF11E5C
:10A13000A114B10421F0D5011196FC92EE9220FFFA
:10A140000FC130E020E090E88FEF12C1C6016DE74B
:10A1500072E143E050E029830E94D15129810097A8
:10A1600031F060E070E0CB01662477240AC0A114CE
:10A17000B10409F4F9C00E5F1F4FF501118300838C
:10A18000F3C03E2D30533A30A0F52260E22FF0E0CC
:10A19000AF014870507022FF07C04115510571F59D
:10A1A0000894611C711C2AC04115510519F00894CE
:10A1B000610871086B017C0152E0CC0CDD1CEE1CC7
:10A1C000FF1C5A95D1F76C0D7D1D8E1D9F1D660FCE
:10A1D000771F881F991F630F711D811D911D68399D
:10A1E000F9E97F07F9E98F07F9E19F0738F0246063
:10A1F00005C03E3F39F423FD3FC02860D801ED90F3
:10A200008D01BFCF353311F03531B1F5F801319102
:10A210003D3211F4206102C03B3241F4D801119665
:10A220003C911197319642E050E002C041E050E08D
:10A2300030533A3020F08F01041B150B1DC040E055
:10A2400050E0BCE040385B075CF4DA01AA0FBB1FAA
:10A25000AA0FBB1F4A0F5B1F440F551F430F511D11
:10A26000319130538F013A3060F324FF03C0509591
:10A2700041955F4F640E751EC22EDD2421FF08C07C
:10A28000A114B10429F001501040F501118300839D
:10A290000E947F497B018C01F3E0CF22DD2433E073
:10A2A000C316D10421F417FB109517F91095C801B6
:10A2B000B70120E030E0A9010E94E248882309F4B8
:10A2C0004AC077FE09C044E9C42E42E1D42E7094FE
:10A2D00061947108739404C03CEAC32E32E1D32E1A
:10A2E00026E0822E912C90E2A92EB12C0FC0F6010F
:10A2F0002591359145915491C801B7010E94354A85
:10A30000E62EF72E082F192F6A187B086A147B0493
:10A3100074F7B594A7940894810891088114910466
:10A3200029F08CEF9FEFC80ED91EF0CFB701C801FE
:10A33000282F220F292F221F2F3F39F020E030E055
:10A34000A9010E94E248882331F482E290E09093D0
:10A35000B4038093B3033E2D2F2D902F812F08C07F
:10A3600030E020E090E803C030E020E090EC8FE7A0
:10A37000F901AC016F2F722F852F942F0F90CF9181
:10A38000DF911F910F91FF90EF90DF90CF90BF90E2
:10A39000AF909F908F907F906F9008959927882716
:10A3A0000895FB01DC014150504088F08D918134CB
:10A3B0001CF08B350CF4805E659161341CF06B35BC
:10A3C0000CF4605E861B611171F3990B0895881B74
:10A3D000FCCFDC0101C06D9341505040E0F708957F
:10A3E000629FD001739FF001829FE00DF11D649F79
:10A3F000E00DF11D929FF00D839FF00D749FF00D05
:10A40000659FF00D9927729FB00DE11DF91F639FA5
:10A41000B00DE11DF91FBD01CF0111240895F8947D
:02A42000FFCF6C
:10A4220028457874507772290000617478707772C9
:10A432006F6B005874616C00496E7465726E0057E0
:10A4420061746368646F67004E6F726D616C004F78
:10A452004E004F4646004F6E004F666600486967E1
:10A4620068004C6F770001010000C841AE47E13C33
:10A47200AE47E13CAE47E13C0AD7A33B0AD7A33B38
:10A48200053333234100009041000058416666665F
:10A49200410000A0400000204100004041CDCC4CD2
:10A4A2003F0A00007A455802050001010000FF033F
:10A4B2008A000400000000000000FF03880005007D
:10A4C200000000001A01011403050001020306073F
:10A4D2000A0B0E0F020306070A0B0E0F2000BA0327
:02A4E200000078
:00000001FF
